:020000040100F9
:1000000038080020E5000001ED000001EF000001CC
:1000100000000000000000000000000000000000E0
:10002000000000000000000000000000F1000001DE
:100030000000000000000000F3000001F5000001D6
:10004000F7000001F7000001F7000001F7000001D0
:10005000F7000001F7000001F7000001F7000001C0
:10006000F7000001F7000001F7000001F7000001B0
:10007000F7000001F7000001F7000001F7000001A0
:10008000F7000001F7000001F7000001F700000190
:10009000F7000001F7000001F7000001F700000180
:1000A000F7000001F7000001F7000001F700000170
:1000B000F7000001F7000001F7000001F700000160
:1000C0000348854600F056F80048004781050001C6
:1000D0003808002040BA7047C0BA70470138FDD1D7
:1000E000704700000448804704480047FEE7FEE7E9
:1000F000FEE7FEE7FEE7FEE795030001C100000111
:1001000030B50B46014600202022012409E00D46AF
:10011000D5409D4205D31D469540491B2546954037
:1001200040191546521E002DF1DC30BD03460B432D
:100130009B0703D009E008C9121F08C0042AFAD29D
:1001400003E00B780370401C491C521EF9D2704723
:10015000D2B201E00270401C491EFBD2704700225F
:10016000F6E710B513460A4604461946FFF7F0FFB6
:10017000204610BD064C0125064E05E0E36807CC7D
:100180002B430C3C98471034B442F7D3FFF79CFF45
:10019000E0070001F0070001F7B5D4B004460E46B1
:1001A00000205390052052900025002700BFEFF358
:1001B00010800090FF21453101A8FFF7D0FF00F02B
:1001C00001FA05462448854218D1012000038442E3
:1001D00002D1002053902AE001204003844202D142
:1001E0004011539023E003200003844203D10120F7
:1001F000400253901BE0529857B0F0BD174885421B
:1002000013D101200003844201D153900FE001205B
:100210004003844201D1539009E00320000384424B
:1002200001D1539003E05298E6E75298E4E705AF16
:100230000137FF2241320A4901A8FFF777FF012069
:1002400000F04FF93146569A5398B84752900098AB
:1002500000F047F95298CFE7C440130085601300BF
:1002600008060001F1B58AB0002009907D20C00089
:1002700008900125AD020027002007907F200690FE
:1002800040240026002005900390200102900020C9
:1002900001903E490A98884206D83D4800686102AC
:1002A00088433B49086006E0394800680121C903DA
:1002B0000843374908607D21C9000A98FFF720FFED
:1002C0007D21C9000090FFF71BFF450100BF3048AA
:1002D00000687F21090288430190200201990843A8
:1002E0002B4908600520FFF7F9FE10E00120FFF719
:1002F000F5FE2748406B02210840002800D007E0A7
:100300000598411C05910899884200D900E0EDE765
:1003100000BF1F48C06B86B2AE4201D9771B00E018
:10032000AF1B0298874203D2E0B20390B8B20290AA
:10033000AE4201D3069400E007940699079840184E
:10034000C005000E04900498A04200D103E0049C74
:1003500009988742BBD800BF0D4800687F21090279
:1003600088430190039800020199084308490860F6
:100370000846406840084000486000BF04484068A4
:10038000042108400028F9D10BB0F0BD0090D00343
:100390000010024010B53E48C0690121090708431A
:1003A0003B49C861812000063A4908633A484861E0
:1003B0003A4808623A48006803218903884338496B
:1003C00008603421374800F073F836480069401C53
:1003D000002803D033480069002817D12C48406812
:1003E0000121090408432A4948600846406807215A
:1003F00009028843264948600846406809150843B1
:10040000234948602848FFF72DFF3FE021488069D5
:100410004409640123480078C006C00E04431D4807
:1004200084611B4800680121C9038843184908609A
:10043000084600687F21090288430446194800697C
:10044000000220431249086008464068012109045F
:1004500008430F494860084640680721090288435D
:100460000B49486008464068091508430849486038
:100470000846006A0D490840054908620846006AB6
:100480000849C968090208430149086210BD000013
:1004900000100240007000400F0800001800020029
:1004A00000100140000000200090D003FF00F8FF82
:1004B00070B504460D462A46214601200003FFF789
:1004C0006BFE70BD02E008C8121F08C1002AFAD1F5
:1004D00070477047002001E001C1121F002AFBD1C4
:1004E000704780F31088704710B501460B68486864
:1004F00042085200180C000401246407A04208D1ED
:100500008A4206D30720C0030818824201D2012084
:1005100010BD0020FCE7000030B502460B4600216C
:10052000C94312E01078521C414000240BE04808F7
:10053000CD07ED0F002D01D0074D00E000256840EC
:100540000146601CC4B2082CF1DB18465B1E002873
:10055000E8D1C84330BD00002083B8ED044672B630
:100560000120C007204305490863206880F30888FC
:1005700000BF6068804700BFFEE7000000700040D9
:100580000D4C0E4D0E49206888420BD1202120468B
:10059000FFF7C2FF216A884204D16068022801D1B6
:1005A0004125AD042846FFF79FFF002802D02846CA
:1005B000FFF7D4FF00BFFEE700400001008000010C
:1005C00011C011CA70B5D2B00024002500BFEFF3EE
:1005D00010800646FF21453101A8FFF7C0FD01ACA0
:1005E00001349822074901A8FFF7A0FD0120FFF779
:1005F00078FFA04705463046FFF773FF284652B004
:1006000070BD00004807000140BA7047C0BA70478B
:100610000138FDD170470000F7B50325AD06286A03
:1006200082B016460C46400840002862286A022123
:1006300008432862286A8007FCD466206860012786
:100640002F61A86AC005FCD5992068602F61A86A4F
:10065000C005FCD5FF209130FFF7DAFFFF230133FF
:10066000AB626846EF60352169602F61A96AC905F0
:10067000FCD5AB62A969EF60C9B205226A602F613F
:10068000AA6AD205FCD5AB62AA690902D2B21143AB
:100690000180C80702D0032005B0F0BDAB626869D5
:1006A000FF210831884368616869C91E0843686191
:1006B00002980002483068600820A860EE602F6150
:1006C000A86AC005FCD5FF200130A8620023F61CF3
:1006D000B0080ED0B2081148006899006054060AAC
:1006E00009194E70060C000E8E705B1CC8709A4281
:1006F000F1D8FF200130A8626869FF2108318843E2
:100700006861686938436861286A800880002862E7
:10071000286A38432862002005B0F0BD8000000C34
:10072000032080064169FF220832914341614269FA
:1007300001210A434261026A920892000262026A3F
:100740000A43026270470000002003218906096AFB
:10075000490849000322920611621146096A0222E1
:10076000114303229206116200BF03218906096A20
:10077000022211400229F8D0D1010322920691628F
:100780000321D1609F2151600121116100BF03212C
:100790008906896AFF22013211409142F7D1032272
:1007A00092069162114688694969FF220832914395
:1007B0000322920651611146496901221143032225
:1007C000920651611146096A890889001162114631
:1007D000096A012211430322920611627047000048
:1007E000F00700010000002038080000D4040001D8
:1080000088AA00205D810001299500018D9400015E
:108010000000000000000000000000000000000060
:108020000000000000000000000000000D9B0001A7
:1080300000000000000000001B810001119B0001F6
:108040006F8100016F8100016F8100016F8100016C
:108050006F8100016F8100016F8100016F8100015C
:108060006F8100016F8100016F8100016F8100014C
:108070006F8100016F8100016F8100016F8100013C
:108080006F8100016F8100016F8100016F8100012C
:108090006F8100016F8100016F8100016F8100011C
:1080A0006F8100016F8100016F8100016F8100010C
:1080B000B19C00016F8100016F8100016F8100019F
:1080C0000348854600F088FB0048004709D70001B7
:1080D00088AA002040BA7047C0BA70470138FDD165
:1080E00070470000084B19680868203080F3098841
:1080F000022080F31488BFF36F8F3FBCAE4608BCEC
:1081000004BC62B618470000D4280020EFF31080AA
:1081100072B6704780F310887047EFF309800E4BFA
:108120001A6820381060F0C044464D4656465F46F7
:10813000F0C008B572B608F06DFC62B60CBC1168F0
:1081400008681030F0C8A046A946B246BB4680F386
:1081500009882038F0C81847D428002004488047F0
:1081600004480047FEE7FEE7FEE7FEE7FEE7FEE71E
:10817000819B0001C180000130B50B460146002003
:108180002022012409E00D46D5409D4205D31D461D
:108190009540491B2546954040191546521E002D15
:1081A000F1DC30BDF0B51FB40646002082B00546B4
:1081B0004024019100901BE0019922460F46304671
:1081C00000F0D4F9049A059B801A994110D3104607
:1081D0001946224600F0BAF9361A8F410197224615
:1081E00001200021009F00F0B1F938184D410090A6
:1081F0002046641E0028DFDC019B00982946324699
:1082000007B0F0BD0549064A08685043054A801882
:1082100008604008704701490860704764290020E1
:108220006D4EC6413930000010B5431A934209D251
:108230008318881803E0401E01785B1E1970521ED7
:10824000F9D210BD03460B439B0703D009E008C9D0
:10825000121F08C0042AFAD203E00B780370401CF6
:10826000491C521EF9D210BDD2B201E00270401C6E
:10827000491EFBD270470022F6E710B513460A46A6
:1082800004461946FFF7F0FF204610BD421C017856
:10829000401C0029FBD1801A704710B5002200E075
:1082A000521C835C8C5CA34201D1002BF8D1D8B264
:1082B000E1B2401A10BDC9B203E003788B4203D08B
:1082C000401C521EF9D20020704730B504460020F1
:1082D000034600E05B1C934203D2E05CCD5C401B94
:1082E000F8D030BD03460A780270401C491C002AB1
:1082F000F9D11846704730B505460020034600E026
:108300005B1C934205D2EC5CC85C201A01D1002CA6
:10831000F6D130BDF0B51FB488B00B990998002490
:1083200048400999C00F490049080991C0070B99B5
:108330000090490049080B9109990898A6460843FE
:108340001CD00B990A98084318D0099801244000C2
:10835000420D4800410D099824050003000B2043FD
:1083600009900B980003000B20430B9050181C49F8
:108370004018002201901446104605E000200146F6
:108380000DB0F0BD032801DA034600E003239C464C
:10839000C11A0AAE0AE05F0008ADED5B4F00F75B63
:1083A0007D430027AA187C41491C5B1E6145F2DD14
:1083B000410004AB5A522104120C0A43240C401C05
:1083C0000828DFDB01980290009970460191009027
:1083D000059B049A0799069800F0E6F8D0E700009C
:1083E0000DFCFFFFF0B50C465C4085B0E40FE407E0
:1083F00003944C000026640859009446490802463C
:108400000296224321D062460A431ED06200570DD5
:108410004A000E032303550D012402462C4924056E
:10842000781B1B0B360B40182343264361460090F4
:108430001C46501AB44103D30098401C009002E03F
:10844000921800985B41002803DA0020014605B02D
:10845000F0BD0020012109050746864611E064466B
:108460001D46141BB54106D36546521BB3417446E5
:1084700007430C43A646CD074008490828439218F5
:108480005B4105460D43EAD11046184313D06046C0
:10849000194650407140084306D06046101AB34157
:1084A00006D20122002306E000220123DB0702E0BE
:1084B0000122D2435310009874460105381C6141D3
:1084C000029C039D0019694100F061F8BFE70000BC
:1084D000FD0300000EB505490291002100910A46F6
:1084E0000B46019100F060F803B000BD33040000BA
:1084F0000EB5054A0292002200921346019200F046
:1085000053F803B000BD0000330400004A00090323
:108510000123090B1B0519430A4B10B5520D9A4252
:1085200002DA0020014610BD064B34339A4203DCC8
:108530009A1A00F01BF810BD034BD21800F006F891
:1085400010BD0000FF030000CDFBFFFF10B5202A87
:1085500004DB0146203A9140002010BD91402023C9
:108560009C1A0346E3401943904010BD10B5202AE1
:1085700004DB0846203AD040002110BD0B46D34012
:10858000D0402024A21A91400843194610BD10B5CE
:10859000002B08DA0024401C614192185B411A4309
:1085A00001D14008400010BDF0B51FB482B00546AF
:1085B0000C0003D0084601F09FFC02E001F09CFC97
:1085C00020300246009021462846FFF7BFFF049B5B
:1085D000059A04460F4618431143084314D0184621
:1085E00010431BD0009840210A1A18460599FFF73E
:1085F000BDFF05460E46009A05990498FFF7A6FFB1
:10860000084305D0012004E02046394607B0F0BDFC
:108610000020C11705430E432C43374300990E98A1
:108620006305401A7905E40A00220C43FD0A0A306A
:1086300002D500200146E9E70105101969410C9CAB
:108640000D9D00196941FFF7A2FFDFE7F0B507466E
:108650000846584087B0C00F049048000E465900A5
:1086600040084908BC1A884105D2384631461E46A2
:1086700017460B4602465800400810434CD0300DB8
:10868000039040055900400D490D0590401A029095
:10869000402872DA18030121000B090508430190F4
:1086A00004980092002805D0019952420020884188
:1086B00000920190029840210A1A01990098FFF750
:1086C00045FF05460C466B4607CB00F097F8C019EE
:1086D0007141039A0E0D0023D71756401A467A406F
:1086E000164344D0049A002A2DD0029A012A039AF4
:1086F00015DC1205C01A914101263605001C714196
:10870000D20F059ED2070093019202962A46234675
:10871000FFF74AFF07B0F0BD38463146FAE71605C5
:10872000224A0F46B218C01AB74101210905001CA0
:108730004F4100187F41114618187941E20F10434C
:108740006D19644113E0E2076D0815436408C20720
:108750001443039A01261205C01A91413605001CE4
:108760007141CE07400830434908C01851412A469C
:108770002346FFF70CFFCDE7FFE7049801224000F6
:10878000C117121A00238B4104983146C417381AB6
:10879000A141EEE730B40124E407634030BC55E763
:1087A00030B40124E407614030BC4FE70000E0FF33
:1087B00010B5002904DB0124E40740428C41214626
:1087C000002B04DB1C460123DB075242A3419942E4
:1087D00000D1904210BD0000064C0125064E05E078
:1087E000E36807CC2B430C3C98471034B442F7D3D2
:1087F000FFF76AFCB42F0101D42F010110B5202A24
:1088000006DBCB170846203A1041C1170B4306E0A0
:108810000B461341D0402024A21A91400843194628
:1088200010BD70B58D180478401CA207920F01D1BD
:108830000278401C231106D10378401C03E006781F
:108840000E70401C491C521EF9D1002B15D0027825
:108850000C268A1A3440401C0C2C03D0A401121B95
:108860009B1C08E004782402121B401CF8E71478D3
:108870000C70491C521C5B1EF9D5A942D3D30020B1
:1088800070BD000003B40148019001BD6D560000A9
:1088900003B40148019001BD6560000003B40148C4
:1088A000019001BDB551000003B40148019001BD24
:1088B000E954000003B40148019001BD995700003C
:1088C00003B40148019001BDED57000003B4014815
:1088D000019001BD1D7C000003B40148019001BD61
:1088E000697E000003B40148019001BDC37F000010
:1088F00003B40148019001BDAF7F000003B40148FB
:10890000019001BDAB52000003B40148019001BDCC
:10891000D37E000003B40148019001BDF58F000033
:1089200003B40148019001BDE1FE000003B4014819
:10893000019001BD250E010003B40148019001BD65
:10894000B143000003B40148019001BD8529000036
:108950001CB50020032103460122920200910190E0
:1089600002A1034808F0D6FB1CBD0000434C49009F
:108970000D8A00011CB5002208210A2008F0C1F868
:10898000104908600020022103464A02009101902C
:108990000DA10F4808F0BEFB0020022103464A0249
:1089A000009101900BA10D4808F0B4FB00200321B9
:1089B0000346012292020091019009A10A4808F0A1
:1089C000A9FB1CBD342900204C45443100000000A7
:1089D000919400014C45443200000000DD940001F8
:1089E0005052494E54000000F597000101480078AC
:1089F0007047000038290020002801D0012100E044
:108A00000021014A11707047382900200EB500245A
:108A10000020029000260027451E6DA003F0E2F919
:108A200000BF0021C94301A802F0C0FE002800D108
:108A3000F7E7002E07D030460026694609798142C3
:108A400000D1EEE700BF012F08D1684600795B280E
:108A500001D1022000E000200746E2E7022F3BD1CF
:108A6000002768460079412817D1681C64490978B5
:108A7000884230DA6D1C284603F0AAF801460090BF
:108A80006048FFF72FFC5F48029903F0DDF8029081
:108A90005C48FFF7FBFB84B21DE068460079422882
:108AA00019D1002D17DB6D1E002D08DB284603F0C1
:108AB0008FF8014600905348FFF714FC02E00020B5
:108AC000504908704F48029903F0BEF802904D4893
:108AD000FFF7DCFB84B2A4E7684600791B2801D1CC
:108AE00001279EE7684600791A280BD10020FFF77E
:108AF00083FF45A003F076F92146424803F0A4F82D
:108B000002908EE76846007909280AD102F09CFE9F
:108B100021463C4803F0C4F80446029402F0A6FE45
:108B20007FE7684600790D2803D0684600790A2857
:108B300022D1684600790D2801D10A2000E00D20DD
:108B4000064602F081FE34A003F04CF900202D49C6
:108B50000855084602F0FAFF002003F09BF8294868
:108B600002F08EFF24A003F03DF902F07FFE002406
:108B700000200290451E2AE068460079082803D0AC
:108B8000684600797F2808D1002C20DD601E84B261
:108B900022A003F027F9029419E068460079202802
:108BA00015DB684600797F2811DA3F2C0CDA68461D
:108BB00002792046611C8CB212490A54012101A895
:108BC00002F068FE029402E015A003F00BF928E71A
:108BD0000D0A434C492072656164792E20547970E6
:108BE00065202768656C702720666F7220636F6D43
:108BF0006D616E64732E0D0A63616969632D3E00B9
:108C000039290020689000200D0A5B6C6F67206F87
:108C100066665D0D0A0000000D0A000008200800CD
:108C200007000000F0B589B005460E4602F066FB6D
:108C300004461D48844201D11CA006E04120800466
:108C4000844201D11BA000E01CA0014622461DA0C9
:108C500002F0E0FF242224496846FFF7E5FA2349A1
:108C60000098884204D022A003F0C8F809B0F0BDF3
:108C700020211D4802F05CFE0899884201D129A0FC
:108C800000E029A007463A4628A0019902F0C2FF59
:108C900032A002A90EC902F0BDFF3CA005A90EC971
:108CA00002F0B8FF00BFE1E7008000014150503101
:108CB000000000004150503200000000554E4B4E65
:108CC0004F574E0072756E6E696E672062616E6BF3
:108CD0003A2025732028626173652030782530386A
:108CE0006C58290D0A0000000040000111C011CA93
:108CF000626F6F7473657474696E673A20696E761B
:108D0000616C69642028626C616E6B206F72206DEB
:108D100061676963206D69736D61746368290D0A09
:108D2000000000006F6B000042414400626F6F74EE
:108D300073657474696E673A206163746976655F00
:108D400062616E6B3D25752C207374727563745F60
:108D50006372632025730D0A0000000062616E6B70
:108D6000313A2073697A653D256C752063726333EF
:108D7000323D30782530386C582076657273696FD3
:108D80006E3D30782530366C580D0A0062616E6B8E
:108D9000323A2073697A653D256C752063726333BE
:108DA000323D30782530386C582076657273696FA3
:108DB0006E3D30782530366C580D0A0070B505468A
:108DC0000E460BA003F01AF800240BE00C206043C1
:108DD0000A4BC01842680C206043195808A002F0E2
:108DE00019FF641C062CF1D308A003F007F870BD2E
:108DF000636F6D6D616E64733A0D0A00FC2D0101A5
:108E00002020252D38732025730D0A006B6579739A
:108E10003A20544142203D20636F6D706C6574654B
:108E20002C2055502F444F574E203D2068697374B5
:108E30006F72792C204374726C2B5A203D206C6F1A
:108E400067206F66660D0A00F8B507460C46032FCB
:108E500003DA25A002F0D2FFF8BD6068007831285F
:108E600006D160684078002802D1284D01260EE026
:108E700060680078322806D160684078002802D106
:108E8000234D402603E018A002F0B8FFE4E721A13B
:108E9000A068FFF702FA002804D13146284602F004
:108EA00007FC19E01CA1A068FFF7F7F9002804D11E
:108EB0003146284602F0F4FB0EE018A1A068FFF747
:108EC000ECF9002804D13146284602F0F9FB03E012
:108ED00005A002F093FFBFE712A0A268616802F04C
:108EE00099FE00BFB8E7000075736167653A206CB2
:108EF0006564203C317C323E203C6F6E7C6F666640
:108F00007C746F67676C653E0D0A0000000C0140C1
:108F1000000801406F6E00006F666600746F67673F
:108F20006C6500006C656420257320257320646FD8
:108F30006E650D0A0000000070B505460C46022D56
:108F40000CDAFFF753FD002801D017A000E017A0AE
:108F50000646314616A002F05DFE70BD12A16068A3
:108F6000FFF79BF9002803D10120FFF745FD0CE036
:108F70000EA16068FFF791F9002802D1FFF73CFDD0
:108F800003E00EA002F03AFFE7E7FFF72FFD00280D
:108F900001D005A000E005A0064631460DA002F074
:108FA00039FE00BFD9E700006F6E00006F666600F3
:108FB0006C6F672069732025730D0A0075736167F4
:108FC000653A206C6F67205B6F6E7C6F66665D0D27
:108FD0000A0000006C6F672073657420746F202591
:108FE000730D0A00F8B5074608F0D4F804467D2151
:108FF000C9002046FFF7C0F805462A46214612A0C0
:1090000002F008FE07F07CFA0546294615A002F09A
:1090100001FE07F045FD054607F03CFD06462B46E0
:1090200032460B21C90212A002F0F4FD1DA002F08D
:10903000E5FE002027490870084607F0CFFB2548C9
:1090400002F0DCFEF8BD0000757074696D653A20B1
:10905000256C75207469636B732028256C752073EB
:10906000290D0A007461736B733A2025750D0A008F
:10907000686561703A20746F74616C2025752042B8
:109080002C206672656520257520422C206D696E46
:109090002065766572206672656520257520420D13
:1090A0000A0000006E616D65202020202020202015
:1090B0002020202020737461746520207072696FF5
:1090C0002020737461636B28772920206E756D0DE5
:1090D0000A0000000891002070B504460D4606A164
:1090E00008A002F097FD0DA002F088FE1848016864
:1090F00018A002F08FFD70BD56312E30302E303169
:10910000000000006669726D776172652076657295
:1091100073696F6E3A2025730D0A00004E33325783
:1091200042303331204672656552544F53202B2014
:109130005541525428444D4129202B204C45442070
:109140002B20434C492064656D6F0D0A0000000020
:109150000000002053797374656D436F7265436C32
:109160006F636B203D20256C7520487A0D0A000046
:10917000486070470168254A114001600021016084
:1091800041608160C1602249884208D12049083984
:1091900049680F2211431E4A083A516035E01C49C4
:1091A0001431884208D11A4908394968F02211431C
:1091B000174A083A516028E015492831884209D1F8
:1091C0001349083949680F2212021143104A083A1C
:1091D00051601AE00E493C31884209D10C490839E6
:1091E00049680F2212031143094A083A51600CE002
:1091F00007495031884208D10549083949680F228A
:1092000012041143024A083A51607047FEFF000001
:1092100008000240002904D0026801231A430260BA
:1092200003E00268014B1A4002607047FEFF000035
:1092300010B50246002000230B681C461440002C89
:1092400001D0012000E0002010BD000010B5002278
:1092500002680D4B1A400C6A8B6823430C69234348
:109260004C6923438C692343CC6923434C6A2343D1
:109270008C6A23431A430260CB6843600B688360A7
:109280004B68C36010BD00000F80FFFF10B5002BBE
:1092900001D0106101E00024146110BD0149486152
:1092A0007047000000040140014600200022074BE7
:1092B0001B680B401A46054B5B690B40002B03D023
:1092C000002A01D0012000E0002070470004014086
:1092D000002120498279002A35D00A4612680368A5
:1092E0009A430B461A600A46526803689A430B4633
:1092F0005A60027951180A6803681A430A60154ACD
:10930000926803689A43134B9A601A46D2680368BE
:109310009A43104BDA604279102A0CD11A469268AF
:1093200003681A430B4B9A601A46D26803681A43C3
:10933000084BDA600DE00749427951180A68036862
:109340001A430A6005E0027951180A6803689A43D3
:109350000A6070470004014070B503460A460021C8
:109360000024002076E001268E40156835402C460A
:10937000002C6ED05568022D02D05568122D20D1D8
:1093800008250D40002D0ED0586A4D07EE0E0F2512
:10939000B5400646AE4330464E07F60E5569B54019
:1093A000284358620DE0186A4D07EE0E0F25B540B0
:1093B0000646AE4330464E07F60E5569B540284383
:1093C00018625568012D08D05568112D05D05568D3
:1093D000022D02D05568122D0BD1586801258D4001
:1093E0000646AE4330461579ED06ED0F8D40284315
:1093F000586018684E000325B5400646AE43304617
:109400001579AD07AD0F4E00B54028431860D868F8
:109410004E000325B5400646AE4330464E009568E3
:10942000B5402843D860986801258D400646AE4374
:109430003046D5688D4028439860D86A4E00012593
:10944000B5400646AE4330464E001569B540284348
:10945000D862491C1568CD40002D84D170BD000034
:10946000054901600F2141610021416081600121B6
:10947000C160002101617047FF3F000081627047B9
:109480008161704742694A404261704700BFFEE710
:109490001CB50F4903C90191009000BF01210D487F
:1094A00002F00EF9FFF7A2FA00280BD0012069465E
:1094B00008700198401C019000231A460648006875
:1094C00007F088FBFF20F53007F018F9E6E7000009
:1094D000EC2D0101000C0140342900201CB50F497E
:1094E00003C90191009000BF40210D4802F0E8F847
:1094F000FFF77CFA00280BD002206946087001981B
:10950000401C019000231A460648006807F062FBE1
:109510007D20C00007F0F2F8E6E70000F42D01011D
:1095200000080140342900207047000010B50020D9
:109530001649086301201649087000201549087073
:10954000154908701548164908600120C0021549E0
:1095500008804F2014490870082014490870FF2023
:1095600013490870487088700720C870002008717F
:1095700048718871C8710F480F49C8610F48086267
:109580000F484862002006F011FE10BD0070004038
:1095900060000020C9000020610000200090D0037E
:1095A0006C000020680000206300002064000020A0
:1095B00008010020E5EE0001C000002055F0000188
:1095C000E5EF0001C206D20E01219140014A11606F
:1095D0007047000000E100E010B50446617800200B
:1095E000205600F01BF8A078002809D00020205653
:1095F000C206D20E01219140074A116000BF0AE065
:1096000000202056C206D20E01219140024A80322B
:10961000116000BF00BF10BD00E100E010B50028E0
:1096200019DA1A4A03071B0F083B9B089B00D25804
:109630008307DC0EFF23A3409A438B071B0E84078E
:10964000E40EA3401A43114B0407240F083CA4085E
:10965000A4001A5118E00E4A03231B02D2188308F3
:109660009B00D2588307DC0EFF23A3409A438B074D
:109670001B0E8407E40EA3401A43054B0324240267
:109680001B198408A4001A5110BD00001CED00E055
:1096900000E100E010B5002819DA1A4A03071B0F91
:1096A000083B9B089B00D2588307DC0EFF23A34096
:1096B0009A438B071B0E8407E40EA3401A43114BF9
:1096C0000407240F083CA408A4001A5118E00E4A0D
:1096D00003231B02D21883089B00D2588307DC0E99
:1096E000FF23A3409A438B071B0E8407E40EA3407D
:1096F0001A43054B032424021B198408A4001A51A1
:1097000010BD00001CED00E000E100E0BFF34F8F52
:1097100003480449C860BFF34F8F00BFFEE7000055
:109720000400FA0500ED00E0F7B5D4B004460E469B
:1097300000205390052052900025002700BFEFF332
:1097400010800090FF21453101A8FEF794FD06F03E
:109750000BFD05462448854218D1012000038442B0
:1097600002D1002053902AE001204003844202D11C
:109770004011539023E003200003844203D10120D1
:10978000400253901BE0529857B0F0BD17488542F5
:1097900013D101200003844201D153900FE0012036
:1097A0004003844201D1539009E003200003844226
:1097B00001D1539003E05298E6E75298E4E705AFF1
:1097C0000137FF2241320A4901A8FEF72DFD012091
:1097D00000F0B7FB3146569A5398B847529000981C
:1097E00000F0AFFB5298CFE7C44013008560130030
:1097F000801501011CB500BF0022D243694608480C
:10980000006807F0F2FA0128F6D102F01DF8684668
:10981000017804A0019A00F035FB02F027F8EBE78D
:10982000342900204C4544257520746F67676C65AA
:10983000642C20636F756E74203D20256C750A00C2
:1098400070B50446002500BF00BFEFF31080054649
:10985000012000F079FB00BF01200006241A2046F9
:10986000054909688847064600BF284600F06CFB9A
:1098700000BF304670BD00000400002010B508484D
:1098800008490860943008490860FF382D380749B6
:109890000860C922920006490938FEF7C5FC10BDD0
:1098A0003D2A002004000020080000200C000020B9
:1098B00064170101F8B504460D461646002700BF9F
:1098C00000BFEFF310800746012000F03DFB00BF12
:1098D00001200006241A324629462046054B1B6803
:1098E0009847009000BF384600F02EFB00BF00985C
:1098F000F8BD000008000020002905D0054A526983
:109900000243044B5A6104E0024A52698243014B0C
:109910005A61704700100240002905D0054A92693B
:109920000243044B9A6104E0024A92698243014B6C
:109930009A6170470010024010B500210022214BAF
:109940005B68042423401946002902D0042906D16B
:1099500002E01D4B036005E01C4B036002E01A4B64
:10996000036000BF00BF174B5B68302423401946DB
:109970000909174B5A5C0368D3404360114B5B687D
:109980000724240223401946090A124B5A5C4368F3
:10999000D34083600B4B5B68E40023401946C90A3F
:1099A0000C4B5A5C4368D340C360064BDB6A1024FF
:1099B0002340002B02D0084B036102E07D23DB0330
:1099C000036110BD001002400090D0030048E80180
:1099D000601701015817010100093D00F1B58AB077
:1099E000002009907D20C00008900125AD020027CD
:1099F000002007907F20069040240026002005903C
:109A0000039020010290002001903E490A9888426C
:109A100006D83D480068610288433B49086006E07B
:109A2000394800680121C9030843374908607D218E
:109A3000C9000A98FEF7A0FB7D21C9000090FEF73F
:109A40009BFB450100BF304800687F210902884325
:109A500001902002019908432B4908600520FEF778
:109A60003DFB10E00120FEF739FB2748406B022147
:109A70000840002800D007E00598411C059108998E
:109A8000884200D900E0EDE700BF1F48C06B86B2F6
:109A9000AE4201D9771B00E0AF1B0298874203D288
:109AA000E0B20390B8B20290AE4201D3069400E057
:109AB0000794069907984018C005000E0490049872
:109AC000A04200D103E0049C09988742BBD800BFA4
:109AD0000D4800687F210902884301900398000225
:109AE000019908430849086008464068400840005A
:109AF000486000BF04484068042108400028F9D1AC
:109B00000BB0F0BD0090D003001002407047000081
:109B100010B5FEF7FBFA044607F042FB002803D01D
:109B200001200007024948602046FEF7F3FA10BD05
:109B300000ED00E001480249086070470090D00342
:109B40000000002010B50D480069401C002803D01B
:109B50000A480069002803D13421084800F09EF823
:109B600006480069401C002803D00448006900280A
:109B700001D1002010BD01482930FBE768290020F1
:109B800010B53E48C0690121090708433B49C86137
:109B9000812000063A4908633A4848613A48086219
:109BA0003A48006803218903884338490860342112
:109BB000374800F073F836480069401C002803D08D
:109BC00033480069002817D12C4840680121090456
:109BD00008432A494860084640680721090288432B
:109BE00026494860084640680915084323494860EB
:109BF0002848FFF7F3FE3FE02148806944096401EB
:109C000023480078C006C00E04431D4884611B48E9
:109C100000680121C90388431849086008460068A4
:109C20007F21090288430446194800690002204345
:109C300012490860084640680121090408430F4999
:109C40004860084640680721090288430B4948607C
:109C50000846406809150843084948600846006AF4
:109C60000D490840054908620846006A0849C96864
:109C7000090208430149086210BD000000100240BB
:109C8000007000400F0800001800020000100140A2
:109C9000682900200090D003FF00F8FF70B504464B
:109CA0000D462A46214601200003FFF73DFD70BD09
:109CB00010B501F09FFD10BDF8B503460024002645
:109CC000009600250020104EB14200D100BF18467A
:109CD0000E06740FCE06F60E00960127009EB740C2
:109CE0003D46012C01D10C3004E0022C01D1103092
:109CF00000E01430002A03D006682E43066002E01C
:109D00000668AE430660F8BD6A090000002905D068
:109D1000828901235B031A43828103E08289024B1B
:109D20001A40828170470000FFDF0000002A03D044
:109D3000838A0B43838202E0838A8B43838270474A
:109D40000246002001235B02994200D100BF138824
:109D50000B40002B01D0012000E0002070470000E4
:109D600070B502460024002300250020124EB142A7
:109D700000D100BF0E06750FCB06DB0E01269E40FC
:109D80003346012D02D19689334006E0022D02D1DF
:109D9000168A334001E0968A33400C120126A64011
:109DA000344616883440002B03D0002C01D001200B
:109DB00000E0002070BD00006A090000F0B589B025
:109DC00005460E4600240020089000BF00BF002773
:109DD000B089002800D000BF2F462C8A20480440BC
:109DE000F08804432C82AC891E480440B088318935
:109DF0000843718908430443AC81AC8A1A48044083
:109E0000B0890443AC8201A8FFF796FD174887424A
:109E100002D10498089001E00398089032689100FC
:109E20001923089A5A431046FEF7A6F907906421B1
:109E30000798FEF7A1F9040121096420414307981E
:109E4000411A069106990901084632306421FEF74D
:109E500093F90007000F04432C8109B0F0BD000006
:109E6000FFCF0000F3E90000FFFC000000380140D4
:109E700001468888C005C00D7047CA05D20D828092
:109E8000704700000FB410B503A9044B044A0298B0
:109E900000F018F910BC08BC04B0184761BF0001FD
:109EA000C40100200FB410B504A9074B02AA0398FF
:109EB00000F008F9044602A9002000F0AAFC2046A0
:109EC00010BC08BC04B0184713A800017CB51546A7
:109ED000024600201C4600290BD0491E0092019129
:109EE000044B6A462146284600F0ECF8009A00210F
:109EF00011707CBDFDA700012021020C01D01021B2
:109F00001046020A01D010460839020901D0104655
:109F1000091F820801D01046891E420801D0881E00
:109F20007047081A704730B47446641E2578641C64
:109F3000AB4204D3635D5B00E31830BC18471D4699
:109F4000F8E780F31088704780F3108870470000AE
:109F5000F0B51FB486B00998089A030D002102439A
:109F600014D05148514A181850430514119801282B
:109F700010981AD0281A401C00264D4F4D490096C3
:109F800001910490002812DA444211E01198012452
:109F900049A3012801D11098C1430698119A846001
:109FA0000360C26041600BB0F0BD4042E4E704468C
:109FB000210500203F4A001C51410391029012E00C
:109FC000E00707D032463B4601990098FEF7A2F918
:109FD0000191009032463B4610461946FEF79AF929
:109FE00006460F466410002CEAD10498039B002813
:109FF000029A0999089806DAFEF78CF9019B009AF3
:10A00000FEF788F905E0FEF7EDF9019B009AFEF7EF
:10A01000E9F904460E460022284BFEF7C9FB03D897
:10A020000020C043014607E00022254B2046314670
:10A03000FEF70CFBFEF76AFA102409E0002C0ADB9D
:10A040000A220023FEF7AEF8079B30321A55641E31
:10A0500002460A43F2D11122641C079B121B1C19F1
:10A06000119B012B03D0012308430ED10AE00843C2
:10A0700004D0112010900020119077E71098151A45
:10A080006D1E0BE01098824202DD00236D1C03E080
:10A09000824201DA00236D1E002BEED00698119942
:10A0A0008260C16030C07EE701FCFFFF104D000000
:10A0B000000014400000F03F300000000000F043BA
:10A0C0000000E03FFFB597B00646002518E22528BE
:10A0D00077D100242746FD49049400E00443761C10
:10A0E00032780120203A90400842F7D130782A286F
:10A0F0000ED00222307801463039092916D8049949
:10A100000A235943303940181443761C0490F1E770
:10A11000189802C804911890002904DA012040031D
:10A1200004434842049002200443761C30782E28D1
:10A1300014D1042004437078761C2A2809D1189879
:10A14000761C80C8189009E00A214F43303FC71998
:10A15000761C3078014630390929F5D930786C28D9
:10A1600010D006DC4C281AD068280ED06A2817D1E7
:10A1700004E0742813D07A2812D110E001204005A1
:10A1800004430CE00121090501E0032109050C430A
:10A190007178814203D1012000052418761C761CB9
:10A1A0003078119066280BD013DC58287DD009DC5C
:10A1B00000287BD04528F6D04628F4D047281AD16D
:10A1C000A5E118E0632835D0642870D0652812D145
:10A1D0009DE170286CD008DC6728F1D069287BD01D
:10A1E0006E280DD06F2806D1BAE073282ED07528BE
:10A1F00071D0782859D01A9A199990476D1C7EE130
:10A200006002400F022809D003280DD004281898B6
:10A2100001680DD00D60001D189070E11898EA17C4
:10A2200001680D604A60F6E7189801680D80F2E752
:10A230000D70F0E718986A4601781172001D1890A9
:10A240000020507202A80090012005E0189802C872
:10A25000189000200091C04361070DD5002101E056
:10A260000199491C0191B94212DA8142F8DB009A46
:10A27000515C0029F4D10BE0002101E00199491C57
:10A2800001918142FADB019A0099895C0029F5D19C
:10A29000019904981A9B471A21463846199A00F0EA
:10A2A00097FA0199401945180BE04FE02CE113E0B3
:10A2B0004EE0009800990078491C00911A9A19996B
:10A2C00090470198401E0190401CF2D1214638462B
:10A2D0001A9B199A10E137E00A20002100900191A1
:10A2E0006002410F022907D0189A01CA1892C217BA
:10A2F0009446032908D00AE01898C01DC108C90077
:10A3000005C91891944607E000B2C2179446042983
:10A3100002D140B2C1178C4600226146944506DA4C
:10A320000A460021404291418C462D2102E0210540
:10A3300004D52B216A461173012103E0E10701D006
:10A340002021F7E7029155E00A200AE0102008E0FA
:10A35000102000900021042004430191082703E00D
:10A3600008200021019100906002410F022907D0CE
:10A37000189A01CA189200229446032908D008E0CE
:10A380001898C01DC108C90005C91891944603E07A
:10A3900080B2042900D1C0B200210291210729D541
:10A3A0001199702906D0009A1021019B4A401A4346
:10A3B00005D00EE040216A461173012108E0614694
:10A3C000014306D030216A4611731199517302215D
:10A3D0000291009A0821019B4A401A430AD1614622
:10A3E000014301D1610705D530216A46117301216E
:10A3F0007F1E02911199582904D035A10E910DA903
:10A400000D910DE037A1F9E76146019B009AFDF738
:10A41000C9FE0E9B8C469B5C0D9A521E0D921370CA
:10A4200061460143F0D10D9805A9081A203001902A
:10A43000600703D501200004844300E00127019850
:10A44000874201DD381A00E0002001990090411890
:10A45000029809180498401A0490E00306D4214693
:10A460001A9B199A049800F0B3F94519002706E0E1
:10A4700003A81A9AC05D199990476D1C7F1C029819
:10A480008742F5DBE0030CD521461A9B199A049804
:10A4900000F09EF9451904E01A9A30201999904766
:10A4A0006D1C0099481E00900029F5DC08E00D980D
:10A4B0000D990078491C0D911A9A199990476D1CB5
:10A4C0000199481E01900029F1DC63E1092801008F
:10A4D000303132333435363738396162636465661A
:10A4E00000000000303132333435363738394142DC
:10A4F000434445460000000000F05AF94519761C17
:10A500003078002800D0E2E528461BB0F0BD600797
:10A5100000D406271898C01DC108C90048680A68F9
:10A520000831C30FDB071891190001D09CA108E086
:10A53000210501D59BA104E0E10701D09AA100E02B
:10A540009AA1430011985B08109165280CD006DC95
:10A55000452809D046281DD0472841D141E066282A
:10A5600018D067283CD13CE00021112F01DB1120DD
:10A5700000E0781C0191009008A911A8FFF7E8FC01
:10A58000139905910021119A15927F1C1298019739
:10A59000009150E00120C00703900120019008A91C
:10A5A000009711A8FFF7D4FC139A14990592002282
:10A5B000119B009212981593059A0192002901D0DF
:10A5C000104602E0791C40180190381A01D5019814
:10A5D00004E04042401E0090781C0190C01B029095
:10A5E00043E0012F00DA01270021112F01DD1120A6
:10A5F00000E038460191009008A911A8FFF7A8FCD7
:10A6000013990591119A00211298159200910197C2
:10A6100021070CD40599B94201DB019900E00191B1
:10A62000012904DD159A491E515C302906D0B84233
:10A6300001DA011D05DA0121029115E00199491E97
:10A64000EDE7002805DC0099411800910199091AED
:10A6500003E0019A411C914200DD01910099401AEA
:10A66000401C02900120C0070390200706D40299E5
:10A670000198814202DB0020C0430290002069461D
:10A68000C87707AF012103980337C907884224D050
:10A69000022011902B201290039800280CDA4042DF
:10A6A00003902D20129007E00A210398FDF764FD26
:10A6B00030317F1E039039701199481E1190002986
:10A6C000F2DC03980028EFD1791E129808703078D8
:10A6D000202108404530BF1E387006A8C01BC01D91
:10A6E000039010980078002800D0012001994118AB
:10A6F0000298C0170918039809180498401A401EB8
:10A700000490E00306D421461A9B199A049800F09D
:10A710005FF8451910980078002803D01A9A199903
:10A7200090476D1CE00324D521461A9B199A049882
:10A7300000F04EF845191CE00098002807DB00994E
:10A740000598884203DD1598405C199901E0199934
:10A7500030201A9A904700986D1C401C0090029877
:10A76000401E0290002804D11A9A2E201999904771
:10A770006D1C0199481E01900029DDDC05E0387848
:10A780001A9A7F1C199990476D1C0399481E0390D3
:10A790000029F4DC21461A9B199A0498ACE60000C3
:10A7A0002D0000002B000000200000000000000031
:10A7B000F8B5044600251E461746880404D405E073
:10A7C00039462020B0476D1C641EF9D52846F8BDD7
:10A7D000FFB50446002581B01E46C80301D53027C9
:10A7E00000E02027880404D505E038460399B047E7
:10A7F0006D1C641EF9D5284605B0F0BD4A68002AD4
:10A8000006D00A68531C0B6010704868401E4860F0
:10A8100070470A68531C0B601070704700B599B000
:10A82000602101A8FDF727FD122108A8C17112229D
:10A8300013A102A8FDF7F8FC002110A8C17100BF08
:10A840000172012141720021C17201218172002136
:10A85000817401210176002116A84180A021818008
:10A86000012110A88177B4211E3041801921C9012E
:10A8700081800848019001A803F0D0F819B000BD0C
:10A88000110610CA000011CA114B008011CA11CA6A
:10A8900011CA000099A80001022804D0032803D09F
:10A8A000042803D101E002E001E000E000BF00BFA6
:10A8B0007047000010B501200649087000F0D2FA78
:10A8C00000F0C2FF0448817804A0FFF7DBFA00F033
:10A8D000CDFF10BD00220020602E00205B424C45C1
:10A8E0005D20636F6E6E65637465642C20636F6EAC
:10A8F0006964783D25750A0010B500200749087085
:10A9000000F0B0FA00F032F900F09EFF04A0FFF76B
:10A91000B9FA00F0ABFF03F0ADF810BD0022002043
:10A920005B424C455D20646973636F6E6E65637452
:10A9300065642C207265737461727420616476653D
:10A9400072746973696E670A0000000010B58CB0FC
:10A950002C2101A8FDF78FFCFFF7F4F80446002C2A
:10A9600005D00622214602A8FDF75EFC04E006227F
:10A9700011A102A8FDF758FC00216846C171C181F0
:10A980000A21817109210174027C0DA11130FDF7AA
:10A990004BFC0C2168468184182101A841840021C8
:10A9A0008184FF21F531C18408496846818501A869
:10A9B00003F07AF90CB010BD010203040506000093
:10A9C00043414949432D4D434D0000008813000089
:10A9D00000B589B000200690079008901D480068D7
:10A9E0001D4909681D4A12681D4B1B68019302929C
:10A9F000039104901B48008800901B4803681B4883
:10AA000002881B4801681B48FFF73CFA1A48069069
:10AA10000020079008A9087006A803F061FAFFF764
:10AA200095FF00F0AFF9FFF7F9FE00F07DF800F0B8
:10AA300083F8124800F0D4F903F01CF8002002213A
:10AA400003460A02009101900DA10E4806F062FB38
:10AA500009B000BD2C010020280100203401002095
:10AA60003001002024010020200100201C010020D2
:10AA700018010020442E0101BDAA0001FDAB000118
:10AA8000424C450061B60001014800787047000063
:10AA90000022002007480078002803D00648008ED6
:10AAA000172801D2112070470348008EC01E80B2C3
:10AAB000F9E7000000220020602E002010B50446B7
:10AAC0002078012806D0022805D0032806D00728C0
:10AAD00011D106E010E0FFF7EDFE0DE0FFF70CFFEF
:10AAE0000AE000F0B1FE0548018E05A0FFF7CAF9A3
:10AAF00000F0BCFE00E000BF00BF10BD602E0020D3
:10AB00005B424C455D204D54552075706461746501
:10AB1000643A2025750A000070B504460D462946A2
:10AB2000204600F0A9F970BD10B5024802F004FFFC
:10AB300010BD0000EDAD0001002006490870064977
:10AB400008800649088006490870064908800649B9
:10AB500008807047CC280020C8280020CA28002080
:10AB6000CD280020CE280020D028002010B50020BD
:10AB700004490880044908700449088000F0ACFBCF
:10AB800010BD0000CE280020CC280020C8280020BE
:10AB900010B518480088002803D0FFF775FF00287B
:10ABA00000D110BD1448C07813490979090208433F
:10ABB000C01D84B20F480088844203DD00200D4987
:10ABC0000880EEE721460C48FFF7A6FF00280FD1CA
:10ABD00008480088001B07490880084600880028AC
:10ABE00006D005480119034802880348FDF71CFBFD
:10ABF00000BFD6E7CE28002037330020F3B583B05E
:10AC0000074600267CE0BC5D40480078002804D060
:10AC1000012810D002286AD132E0CA2C0AD13C485F
:10AC2000047001203B49088005203B490880012031
:10AC30003649087061E0374801880088401C354A71
:10AC400010803348445410460088052817D13049F5
:10AC5000C9782F4A1279120211430846FF21E131C7
:10AC6000884205DD0021294A11702A4A118005E039
:10AC7000C11D294A11800221244A117000BF3CE005
:10AC8000244801880088401C224A108020484454EF
:10AC90001046008820490988884227D11C48C0787E
:10ACA0001B490979090208430546E81C81B2184886
:10ACB000401C04F099FA0290681D1549095CA81D12
:10ACC000134A105C000201430191019902988842E5
:10ACD00005D1917850782B46521D04F0ABFA002034
:10ACE0000A49087000210B48018000BF05E00020E0
:10ACF000064908700749088000BF00BF701C86B273
:10AD00000498864200DA7EE705B0F0BDCC2800202A
:10AD10003C300020C8280020CA280020FFB581B0A0
:10AD200006460F461C46E01D80B200900098FB28A6
:10AD300003DD0020C04305B0F0BDCA2010490870F3
:10AD4000084646708770CC7020120871002C05D020
:10AD500022460B48401D0399FDF766FAE01C81B2BC
:10AD60000748401C04F040FA0546601D044A15548B
:10AD70002912A01D11541046009904F099FADAE73F
:10AD80003C32002000B587B01C216846FDF773FAFD
:10AD900000216846017310480290052168468170C1
:10ADA000032101701021C170002141700171012146
:10ADB0004171002181714173084805900521684661
:10ADC00081737D210901018200200690684603F00D
:10ADD0008DFD07B000BD000040E2010000800701CA
:10ADE00010B50446204600F07FF810BD70B514235E
:10ADF000032207210D480CF49FD604461B20207027
:10AE000000206070472060800320A0800020E08048
:10AE100025460835064868600648A860072028705F
:10AE200020460CF4C5D600F007F870BD1B0D0000DD
:10AE3000302D0101202D01011FB5472168460181F8
:10AE40000648039002A803F007F8472168460180EE
:10AE500003480190684604F0E3F81FBDE42D0101AA
:10AE6000ADFE0001002002490870024908707047D9
:10AE7000C0280020C1280020F8B506460D46164817
:10AE80000078002803D015480078002802D0002060
:10AE9000C043F8BD472004F0DDF80746A81D83B283
:10AEA000032239460E480CF447D604460D488078F4
:10AEB00020700120607005206080A5802A46314600
:10AEC000A01DFDF7B1F920460CF472D6012003490C
:10AED00008700020DDE70000C0280020C128002005
:10AEE00006470000602E00200149086070470000FE
:10AEF000C4280020F8B504460D4616461F460248F1
:10AF000003F010FA0020F8BD042F002010B53E48D1
:10AF10000079002877D12C23032207216D204001DE
:10AF20000CF40AD60446A02020703848C07860701F
:10AF3000002020710321E1800021617201216171F3
:10AF400007212177324881796177407B002804D03E
:10AF50000021E1800321617117E02D48C0790028AC
:10AF600013D02B488079022801D10121617701207B
:10AF700020710121E180264881792120015501219C
:10AF8000222001550021202001551F4880790228E8
:10AF900004D003281FD004282BD123E003F096FC13
:10AFA00000280ED00521E1800021617118480E3083
:10AFB000818861618188A16120460A3003F0BDFA71
:10AFC00008E00320104988711148143081886161BC
:10AFD0008188A1610EE00E4814308188616181880A
:10AFE000A16107E00A481A30818861618188A16106
:10AFF00000E000BF00BF01200349087148712046EE
:10B000000CF4D6D500BF10BD602E0020E42E002029
:10B01000502F002010B502230322072120480CF4F2
:10B020008BD50446A72020701E48C078607006208B
:10B030001C4948710020087103200CF43BD60328FA
:10B0400003D105201749887126E016488079012828
:10B0500006D0022805D003280CD0042817D112E00E
:10B0600000BF1148007D002803D003200D498871DE
:10B0700011E000BF0C48807E002803D0042009495D
:10B08000887108E000BF05200649887103E00520AB
:10B090000449887100BF00BF20460CF489D510BD5B
:10B0A000A30D0000602E0020502F0020FEB50446A6
:10B0B0000D4616461F4601A83B46324629460090DB
:10B0C000204603F043FC68460079002800D1FEBD0D
:10B0D00001A83B46324629460090204600F0C2F8BF
:10B0E00068460079002800D1F1E70548406C002847
:10B0F00004D003482946426C204690470020E6E7EA
:10B10000602E0020FFB583B004460D4626791AE074
:10B11000F10020684018083803C802910190684681
:10B120008088A84204D0684680880949884208D1AE
:10B1300003222846029F069B0599B847C0B207B074
:10B14000F0BD701EC6B2002EE2DC0020F7E7000062
:10B15000FFFF0000F8B504460D4616461F4603F0F3
:10B1600093F805480069002803D0034801690420CA
:10B1700088470020F8BD0000702F0020F8B5064673
:10B180000F463148406BC007C00F002833D02E480F
:10B19000856B2E4800687E2148432C1A2C48008875
:10B1A000401E2B4908802B48844202DB40428442E7
:10B1B00020DD0020264908802348006A400840001E
:10B1C00021490862244800680321890308400028B7
:10B1D00005D02148006888431F49086006E01E48E2
:10B1E00000680321890308431B4908601B49487F05
:10B1F00002F0D2FD00BF1648008800280BD012488C
:10B20000006B0121084310490863052203211448FB
:10B210000CF454D715E00C48006BFF210902884359
:10B22000094908630846006B05218902084306495D
:10B2300008630846006B012108430349086303F0D3
:10B2400075FB0020F8BD0000001002408C000020BB
:10B2500082140020A8FDFFFF00100140C02E002036
:10B26000010F0000FFB581B004460E4627120020F2
:10B2700000900E2F0ED11548844223DB134809306D
:10B2800084421FDC324621461148049BFFF73AFFF7
:10B29000009017E0002510E0E9000E48405AB8423F
:10B2A00009D1EA000B495118486832462146049BEF
:10B2B000FFF728FF0090681CC5B20648001F007801
:10B2C000A842E9DC009805B0F0BD0000120E0000B5
:10B2D000C4290101102E00200020044908700449EF
:10B2E000086004490860044908607047402900204C
:10B2F00054290020582900205C290020004870476C
:10B3000000800001F8B504460D4616461F46102C75
:10B3100004D0112C08D0122C12D10BE03A46314641
:10B32000284603F06BFB0CE03A463146284603F012
:10B33000DDFB06E03A463146284603F06BFC00E0B0
:10B3400000BF00BFF8BD10B50446002010BD0000CE
:10B3500010B501230322072104480CF4EDD3044661
:10B360000120207020460CF423D410BD020D0000F3
:10B3700070B51E48C079002802D01C48057B02E049
:10B380001A482038C5782B1D0322072118480CF4D1
:10B39000D3D30446A92121701648C17861700021D9
:10B3A00061801248C079002807D01048027B4038DD
:10B3B000816C201DFCF738FF07E00C482038C2786C
:10B3C00001461C39201DFCF72FFF60884019608062
:10B3D00008480079062802D0022006490871022098
:10B3E0000449487120460CF4E3D370BD502F00206F
:10B3F000A60D0000602E0020F8B51F26232303228F
:10B40000072131480CF498D30446AA2020702F4815
:10B41000C07860702E48C07860802D48C2780146A0
:10B420001C39201DFCF700FFA078301AC6B26188D5
:10B43000201D0D18032E14DD25480079002810D09A
:10B440000320287019206870224840890012E87093
:10B450002048807AA8706088001D60802D1D301FF4
:10B46000C6B2022E21DD1A48407900281DD0194AA3
:10B47000107BB11E884201D2024600E00A46D7B2D4
:10B48000781C28701348007BB84201D1092000E0E5
:10B49000082068703A460F490D31A81CFCF7C4FE1D
:10B4A0006188B81C0818608000BF08480079062829
:10B4B00002D0032005490871032004494871204641
:10B4C0000CF476D3F8BD0000A60D0000602E00201D
:10B4D000502F0020E42E002010B53A23032207212C
:10B4E0001C480CF429D30446A42020701A48C078C4
:10B4F000607019488079022804D0032808D00428F5
:10B5000014D10CE01548408864214843608010E065
:10B510001248801D408864214843608009E00F483C
:10B520000C30408864214843608002E00020608045
:10B5300000BF00BF0021217108490E39887901F050
:10B54000F1FF0520044908710420487120460CF4DD
:10B550002FD310BDA10D0000602E00205E2F002013
:10B5600010B502230322072108480CF4E5D2044653
:10B57000A52020700648C078607007200449087133
:10B580000520487120460CF413D310BDA20D000015
:10B59000602E0020FFB583B00C46154600200190B8
:10B5A000029001A90398FDF76DF90746002F50D1CD
:10B5B0000521C90201A8FDF76BF9002827D126490A
:10B5C00001A8FDF765F9002821D12349891C01A8AC
:10B5D000FDF75EF900281AD11F49491C01A8FDF7A3
:10B5E00057F9002813D12921090201A8FDF750F9C4
:10B5F00000280CD1194901A8FDF74AF9002806D105
:10B600001649491C01A8FDF743F9002801D0062777
:10B610001FE0019880880121C9030840C013002859
:10B6200016D1019881880905090D46187088A8422D
:10B6300000DA072760193188884201DD0D2706E00E
:10B64000311D481922460699FCF7EEFD748000E092
:10B650000627384607B0F0BD012800000229000087
:10B6600000BF1FF49DD6FFF793FA012005F046F8BE
:10B67000F7E7000010B50121074801F02DFF402138
:10B68000064801F029FF0121034800F009F8402194
:10B69000024800F005F810BD000C01400008014010
:10B6A00070B504460D4629462046FDF7E7FE70BDFD
:10B6B00070B504460D4629462046FDF7E1FE70BDF3
:10B6C00070B504460D4629462046FDF7DBFE70BDE9
:10B6D00000B58BB001210820FEF71EF90121880377
:10B6E000FEF71AF905A8FDF7BBFE402005900220E1
:10B6F000069004200A9005A92648FDF72DFE80201B
:10B70000059004200A9005A92248FDF725FEE120B6
:10B7100040020190002168460181418181810182BE
:10B720000C21C18101A91C48FEF748FB01210846F4
:10B73000FEF7E2F81948FDF71DFD0123174A1749E6
:10B7400008390220FDF7A2FD012280211248FEF7F0
:10B75000EDFA00220121402005F0D3F910490860DC
:10B76000012005F0BFF90F49086001220E490A487F
:10B77000FEF7A2FA1C2168460170032141700121E5
:10B780008170FDF729FF01210348FEF7BFFA0BB0D6
:10B7900000BD0000000C01400038014008000240DC
:10B7A0002C290020302900202505000070B5054611
:10B7B0000C460F480068002800D170BD601C0028AE
:10B7C00001D1401E07E07D21C900614308467D216B
:10B7D000C900FCF7D1FC06463246294604480068F9
:10B7E00005F003FB012800D1E7E70020E5E70000B2
:10B7F0002C2900201CB5002001900F490F48FEF7AE
:10B80000AFFA002817D00D48FEF732FBC0B2009007
:10B810000B480068002806D0002301AA69460848A2
:10B82000006805F084FA0198002803D00120000781
:10B830000449486000BF1CBD2505000000380140D8
:10B840002C29002000ED00E010B507480068002812
:10B8500008D005F08DFC022804D1C11E0248006802
:10B8600005F05FFB10BD00003029002010B508482E
:10B87000006800280AD005F07BFC022806D10023CE
:10B880001A4619460248006805F0A4F910BD0000E8
:10B890003029002030B58BB004460D46002C01D075
:10B8A000002D01D10BB030BD00211F48FDF7B2FCC7
:10B8B0001D4908390220FDF75BFC1C4800900194EB
:10B8C0001020029003950020049080200590002015
:10B8D00006900790089003200003099000200A902A
:10B8E00069461148FDF7B2FC01210F48FDF792FCB3
:10B8F00000BF0D4908390220FDF79AFC0028F8D056
:10B9000000210948FDF786FC074908390220FDF7A8
:10B910002FFC00BF40210548001FFEF711FA002848
:10B92000F8D000BFBEE70000080002400438014024
:10B9300030B502460B460021C94312E01078521C74
:10B94000414000240BE04808CD07ED0F002D01D049
:10B95000074D00E0002568400146601CC4B2082C79
:10B96000F1DB18465B1E0028E8D1C84330BD00005B
:10B970002083B8ED70B504460A2C17DAA0000C49F4
:10B980000858002812D0A0000D580A4885420CD053
:10B990000948854209D00020A100054A5050A10065
:10B9A000064A50502E462046B04700BF70BD0000EA
:10B9B000EC2F0020D7040101D50401011430002030
:10B9C000F8B507460C4620780A2824DA2578A8001E
:10B9D000124908581249884207D10020A9000F4A8D
:10B9E0005050A9000F4A505014E0A8000B490858C5
:10B9F0000D4988420ED10823032211460B480CF44E
:10BA00009BD00646207830706068706030460CF439
:10BA1000CFD000BF00BF0020F8BD0000EC2F0020F9
:10BA2000D504010114300020D7040101060F0000E5
:10BA300010B503460A46002000219488022C01D04C
:10BA40000D200DE0D188002B05D0002908D0012958
:10BA500006D0812004E0002902D0022900D08120F4
:10BA600010BD0620704700000146062904D20C20B4
:10BA70004843024A105870470020FCE7FC2D0101A2
:10BA8000F0B589B0074600263C4621E000E0641C82
:10BA900020782028FBD020780928F8D020780028AA
:10BAA00000D11AE03046761C800001A90C5000E05D
:10BAB000641C2078002805D02078202802D0207827
:10BAC0000928F5D12078002802D000202070641CBD
:10BAD0002078002801D0082ED8DB00BF002E02D12C
:10BAE000002009B0F0BD002513E00C226A430D4B85
:10BAF00099580198FCF7D1FB002809D10C20684324
:10BB00000849401801A98268304690470020E8E7BC
:10BB10006D1C062DE9D304A0019900F07BF80120EB
:10BB2000DFE70000FC2D0101756E6B6E6F776E20F4
:10BB3000636F6D6D616E643A20257320287472798D
:10BB4000202768656C7027290D0A000070B504462F
:10BB50002078002800D170BD1A480078002813DD35
:10BB600019490978C81DC117490F0918C910C9001A
:10BB7000411ACDB2A901154A88182146FCF78DFB60
:10BB8000002800D1E7E700BF0F49097889010F4A73
:10BB900088182146FCF7A6FB0B490978481CC117F9
:10BBA000490F0918C910C900411A074A1170054800
:10BBB0000078082804DA03480078401C014908701E
:10BBC00000BFC8E7392900203A290020688E0020EC
:10BBD0000146084B1B785B1E5B1A18460830C317DA
:10BBE0005B0F1B18DB10DB00C21A9001024BC01860
:10BBF000704700003A290020688E002070B5044686
:10BC00002046FCF743FB85B229462046FFF742FE5B
:10BC100070BD00000FB408B503A80090602109486A
:10BC2000009B029AFEF752F900200090002105487F
:10BC30004030C177403800F0E1F801B008BC04B0F2
:10BC400018470000A8900020F8B507460D46384672
:10BC5000FCF71CFB84B20BA000F0C4F8002604E043
:10BC60000BA000F0BFF8701C86B2AE42F8DB05A056
:10BC700000F0B8F8002C03DD21463846FFF70AFE35
:10BC80002046F8BD0D63616969632D3E0000000028
:10BC90002000000001490860704700003C29002096
:10BCA000F0B593B006460C46002500200290FFF741
:10BCB000D8FE0190224620213046FCF7FCFA0028ED
:10BCC00002D0204613B0F0BD00203055002729E0F7
:10BCD0003846FFF7C9FE0090224631460098FCF72F
:10BCE0000AFB00281DD10298002808D103A800995A
:10BCF000FCF7F8FA03A8FCF7C9FA85B20EE001E0F8
:10BD0000681E85B2A54206DD2A4603A80099FCF705
:10BD1000F2FA0028F4D1002003A948550298401CEB
:10BD200002907F1C01988742D2D30298002801D14B
:10BD30002046C7E70298012819D109E003A908198C
:10BD40000121FFF7A7FD03A8005D3055601C84B2F8
:10BD50003F2C01DAAC42F1DB3F2C06DA20203055D3
:10BD6000601C84B21CA000F03DF82046AAE7A54262
:10BD70000FDD09E003A908190121FFF78BFD03A8D6
:10BD8000005D3055601C84B23F2C23DAAC42F1DBFD
:10BD900020E012A000F026F8002711E03846FFF757
:10BDA00063FE0090224631460098FCF7A4FA002872
:10BDB00005D1009800F016F809A000F013F87F1CD8
:10BDC00001988742EAD305A000F00CF821463046DE
:10BDD000FFF73AFF204675E7200000000D0A00003B
:10BDE0002020000070B504462046FCF74FFA85B2CB
:10BDF00029462046FFF74EFD70BD000010B50446F1
:10BE000006480068002804D020460449096888478D
:10BE100002E02046FFF7F2FE10BD00003C290020A2
:10BE200030B504460020014D287030BDC1280020E7
:10BE3000F8B507460C466588A688022D13D0062D56
:10BE40001BD1022E0ED1A279E1795018012803D11D
:10BE500001210C4A117004E0002802D10021094A96
:10BE6000117000BF0AE008480068002804D0A188CB
:10BE7000A01D054A1268904700E000BF00BF0020E7
:10BE8000F8BD0000C0280020C4280020FFB581B004
:10BE90000E461F4600250FA0009005252B460833AF
:10BEA00039460E48039A0BF447D604460020A07189
:10BEB00030782070A58070886080002D04D02A46DC
:10BEC000E01D0099FCF7B0F920460BF471D6002074
:10BED00005B0F0BD4341494943000000054700005B
:10BEE00010B5FCF78FF910BDF8B507463E46002E99
:10BEF00002D172B600BFFEE714480068864201D145
:10BF0000002420E004F08CFB756904F097FB1048D6
:10BF10000068854203D00F480068854201D10224A1
:10BF200011E00D48854206D1B06A002801D10324F2
:10BF300009E0022407E00948854201D0002D01D123
:10BF4000042400E001242046F8BD0000D42800208D
:10BF5000D8280020DC28002054360020403600205D
:10BF600070B504460D460A2C0AD10D210B48FDF789
:10BF700084FF00BF80210948FDF7E2FE0028F9D0C8
:10BF8000E1B20648FDF779FF00BF80210348FDF7C5
:10BF9000D7FE0028F9D0204670BD000000380140CF
:10BFA000FEB505460C4616461F462078801E030047
:10BFB000FDF7B9FF060438744D73547401203949F4
:10BFC0000870A17838484176A078C007C00F0028D3
:10BFD0000AD00622354934481330FCF725F9334896
:10BFE0000938017A304881742E48808A002809DD9A
:10BFF000FF20F5302B4948800846828A03212C48CF
:10C000000CF45CD02748C06900280AD000200090BA
:10C0100001900520694608702248C1696846884732
:10C0200000BF3CE000212048417601F0F7FD1D48AB
:10C03000C06900280AD000200090019006206946BF
:10C0400008701848C1696846884700BF27E0172272
:10C05000A11C1548801FFCF7E7F820E013480938B9
:10C060008078010111483F300818807B002813D1E7
:10C070001C22A11C0C482038FCF7D6F808222146C7
:10C08000143109481038FCF7CFF8608A0649203986
:10C090000883217F0448417401E000E000BF00BF35
:10C0A0000020FEBDCC2F0020B02F0020692E0020E4
:10C0B000040F0000F0B585B00D461E462223032272
:10C0C00031468B480BF438D504460120607028783F
:10C0D0000300FDF728FF0B07F7F7F7837DEA2AF740
:10C0E000F780F7000120207060708248817921710B
:10C0F0000079A0707F48C17961714179E170017A5E
:10C10000A171417AE171817A2172C06900280BD056
:10C11000002002900390022069460872039475483B
:10C12000C16902A8884700BFDCE007202070012019
:10C13000607068461FF492D20199009803910290B2
:10C14000FFF7CEFE029940186082002710E0FFF74B
:10C15000C7FE02994018C1B2A01CC155FFF7C0FE2E
:10C1600003994018C1B220461430C155781CC7B29B
:10C17000082FECDB08270AE0FFF7B2FE039940180E
:10C1800002994018C1B2A01CC155781CC7B2102F2B
:10C19000F2DB102121775848807801015648483059
:10C1A0000818807B012812D11C22A11C5348FCF7DF
:10C1B0003BF808222146143150481030FCF734F87F
:10C1C000608A4E490883217F4C482030417489E0C1
:10C1D0000520207086E00A20207083E00420207073
:10C1E0006878012802D06878002842D10120607068
:10C1F0004048007C002812D001A81FF42FD2FFF77E
:10C200006FFE3F490090FBF7B7FF3E4808180199C1
:10C2100047183D493846FBF7AFFF039102E0354828
:10C22000C06803903348C06900280CD000200190FA
:10C23000029003206946087103A802902D48C16945
:10C2400001A8884700BF1021A01CFCF714F8039830
:10C25000A070FF21090203980840010AE170FF2144
:10C26000090403980840010C21710398010E6171C3
:10C270001AE06878022817D11E48C06900280AD041
:10C280000020029003900420694608721948C16991
:10C2900002A8884700BF00BF20460C3807460BF4B1
:10C2A0007DD4002005B0F0BD1CE0062020701748AA
:10C2B000C078012807D110220F490F31A01CFBF7CD
:10C2C000B3FF04E00DE01021A01CFBF7D4FF062211
:10C2D0000E49091D20461230FBF7A6FF00212176EA
:10C2E00000E000BF00BF20460BF462D40020D9E775
:10C2F000140E0000CC2F0020602E0020902F002074
:10C30000A0BB0D00A08601003F420F00E42E0020DC
:10C31000FEB505460C4616461F461448006C00281C
:10C320000CD0002000900190029005206946087012
:10C3300001940E48016C6846884700BF20780928A0
:10C340000AD004DC03280BD004280AD107E00C280B
:10C3500004D0142805D100E000BF03E002E001E0B2
:10C3600000E000BF00BF0020FEBD0000602E0020E6
:10C37000FEB507460C461D46FF2D20D01A48006C1E
:10C3800000280CD000200090019002900620694601
:10C39000087001941448016C6846884700BF032068
:10C3A0000BF488D403281DD10F48806F002819D0C2
:10C3B0000D480321826F0D480BF480D612E00A4825
:10C3C0006030007F00020146083101230322074844
:10C3D000001F0BF4B1D306460720307030460BF433
:10C3E000E7D300BF0020FEBD602E0020090E000034
:10C3F000FEB50C4616461F463804000E5E4988708E
:10C4000008468078FF2871D00846807800020146EF
:10C4100008313423032259480BF48ED3054656487D
:10C420008178807802015448483010188170218842
:10C43000514880780201504848308152617A48382A
:10C44000807802014C4848301018C1704A498978F8
:10C450000A01494948315118081D062221460A316E
:10C46000FBF7E2FE207C012808D1012142488078B8
:10C47000020141484830101881730AE0207C0028EE
:10C4800007D100213C48807802013B484830101811
:10C490008173208838490880607A08720622214614
:10C4A0000A3135480930FBF7BFFE02F00FFA0028C9
:10C4B00022D0607A012805D1032211462F48ED3899
:10C4C0000BF48AD302F00CFA0300FDF72CFD0508EB
:10C4D000090A040B10000121282041550BE000BF80
:10C4E00000BF00BF05212820415504E03FE00021A6
:10C4F0002820415500BF02E000212820415503219A
:10C5000030460BF4E9D317201B49088617211A4837
:10C510008078020118484830101841811848C068D6
:10C52000002803D0032117480BF428D51648008DA6
:10C53000002806D01448028D03211248401E0BF437
:10C54000BDD50D48006C00280DD000200090019052
:10C550000290022069460870019402950648016C19
:10C560006846884700BF28460BF422D301E001F05B
:10C5700081FA0020FEBD0000602E0020020E0000A7
:10C58000702F0020030F0000E42E0020FEB50646A9
:10C590000C4617461D46FF212804000E02011648CE
:10C5A0001018817001F0B8FB002803D1022103208C
:10C5B0000BF492D310484838006C00280DD00020AE
:10C5C00000900190029003206946087001940A4887
:10C5D0004838016C6846884700BF10210648293852
:10C5E000FBF749FE05480068002802D009200BF43B
:10C5F0005DD10020FEBD0000A82E0020100C002000
:10C60000FEB504460D4616461F460848C069002878
:10C610000AD0002000900190092069460870034864
:10C62000C1696846884700BF0020FEBDCC2F0020AE
:10C63000F0B591B00D461F461223032239464648F5
:10C640000BF47AD204460020207044480078002879
:10C650004BD04248407C00282FD0002010903C2135
:10C6600001A8FBF708FE01F0F7FE1090109E20E0F5
:10C67000711EC8B201A901F033FF6846808B29887A
:10C68000884208D10822A91C05A8FBF71EFE002835
:10C6900001D1012020702078002808D008A8407D12
:10C6A0006074102201A9601CFBF7BEFD03E0701E40
:10C6B000C6B2002EDCDC00BF17E02948008B2988B9
:10C6C000884212D10822A91C25481030FBF7FDFD35
:10C6D00000280AD10120207021482030407C60745D
:10C6E00010221F49601CFBF79FFD207800281ED1F7
:10C6F0001A48C06900280AD000200F901090082026
:10C7000008A908771548C1690FA8884700BF022308
:10C7100003223946104814380BF40ED20646012085
:10C7200030700620707030460BF442D20EE00B4899
:10C73000C06900280AD000200F901090072008A997
:10C7400008770648C1690FA8884700BF20460BF448
:10C750002FD2002011B0F0BD180E0000CC2F002009
:10C76000902F0020F8B50D4617461E462878002861
:10C7700004D0012819D002283ED126E01C233A46D5
:10C7800031461F480BF4D8D10446287820701D4844
:10C79000007B60801B48027B01460D31201DFBF7AA
:10C7A00043FD20460BF404D227E00A233A463146E3
:10C7B00013480BF4C1D104462878207011484089F1
:10C7C000608020460BF4F4D117E00A233A46314644
:10C7D0000B480BF4B1D10446287820700948008C2E
:10C7E00060800848418CA180818CE180C18C2181CE
:10C7F00020460BF4DDD100E000BF00BF0020F8BDF3
:10C800000B0E0000E42E0020F8B505460C46164637
:10C810001F46207800F086FE0020F8BD70B5044663
:10C820000888064D68860D881804000E0601034826
:10C83000483030188581002070BD0000602E002037
:10C84000FEB507460E461D462804000EFF2828D0D8
:10C850002804000E00020146083106230322E120CD
:10C8600000010BF469D10446012020700220608091
:10C87000FF204130A0800D48006C00280DD0002022
:10C88000009001900290042069460870019602947D
:10C890000648016C6846884700BF20460BF488D1E3
:10C8A00001E001F0E7F80020FEBD0000602E00204E
:10C8B000FEB505460C4616461F460948006C002882
:10C8C0000CD000200090019002900820694608706A
:10C8D00001940348016C6846884700BF0020FEBDF4
:10C8E000602E0020F8B50C4617461E4602233A4635
:10C8F00031460B480BF420D10546A078094908734E
:10C900006288211D07480D30FBF78EFC00206870FF
:10C910002078287028460BF44BD10020F8BD000089
:10C920000D0E0000E42E002030B5044648780028A3
:10C9300007D10C480079012812D10878094DE87018
:10C940000EE04878012804D10D780648203005759E
:10C9500006E04878022803D10D780248203045755A
:10C96000002030BD602E0020F8B505460C46164666
:10C970001F466078002809D11848007906282AD176
:10C9800007201649087101F009F824E060780128B1
:10C9900013D112482030007DFF281CD001F020F96F
:10C9A000FF210E48203001750D480069002812D083
:10C9B0000B480169002088470DE0607802280AD101
:10C9C00006482030407DFF2805D001F0E7F8FF2120
:10C9D0000248203041750020F8BD0000602E002084
:10C9E000702F0020F8B506460C4617461D46032D4D
:10C9F00005D10748017A093001F028FE05E0102230
:10CA0000A11D03481F30FBF70FFC0020F8BD0000FC
:10CA1000602E0020F0B58DB006460D462878A1287E
:10CA20007ED010DC1B287CD006DC012815D0032822
:10CA300078D0172877D197E1282875D0912874D01D
:10CA4000A028F7D1A2E1A2380300FDF76CFA09F49F
:10CA50006CF3F26CF1F0EFEE6C006878002879D19D
:10CA6000012002F015FB01F055FE342303220721BB
:10CA7000FA480BF461D0044603202070F84880780F
:10CA800060700120E076FB206084F648E084F64880
:10CA9000A084F348008820840020A0760622F04974
:10CAA000091D201DFBF7C0FBED48407AC02108405E
:10CAB000C02809D1EA48807805210840002803D120
:10CAC000A07E01210843A076A07E04210843A07621
:10CAD000E6486080E248C078012806D11022E44987
:10CAE00020460A30FBF7A0FB04E0102120460A3064
:10CAF000FBF7C1FBDE480F38006C00280ED0002089
:10CB00000A900B900C90012008A908720B950C94C8
:10CB1000D7480F38016C0AA8884700BF012006E0FB
:10CB20008AE100E117E0D0E186E058E012E000F091
:10CB3000F9FC20460BF43CD0012303220721C7480F
:10CB400015300AF4F9D707461A20387038460BF426
:10CB50002FD000BFBAE1282103A8FBF78CFB0020EF
:10CB60000190029001F0B2FE002805D003A801F068
:10CB700001FD01A801F0C6FC01F0A8FE00280CD0C0
:10CB80006846807C002808D16846807A002804D056
:10CB9000012103A801F0D4F820E00622B049091DC4
:10CBA00003A8FBF741FB0020694688741022B049B6
:10CBB00005A8FBF739FBAA48C078012805D1102247
:10CBC000AB4909A8FBF730FB04E0002009900A906C
:10CBD0000B900C90012103A801F0B2F876E1A44873
:10CBE0001130C07B00281BD11123032207219B4851
:10CBF0001F300AF4A1D70446282020709848C07836
:10CC0000012805D110229A49601CFBF70DFB03E0B7
:10CC10001021601CFBF72FFB20460AF4C9D700BF88
:10CC2000002193481130C17350E1B1E0AFE0F7E06B
:10CC3000ABE0AEE0A8E02EE1012002F029FA0121EC
:10CC400003200BF449D0002401208A4948841F2086
:10CC50000C9083480088402108408011002803D0B0
:10CC600060210C9808430C907D488078052108408D
:10CC7000002804D0FF2181310C9808430C9078489B
:10CC80000088FF21013108400012002804D0032150
:10CC900049020C9808430C90012077490822002390
:10CCA00000930192029103900B230CAA0321C90265
:10CCB00070482230FBF7F2FD0446002C00D005E15D
:10CCC00000206E498886FF200B9001206C490622C7
:10CCD0000023009301920291039008230BAA694953
:10CCE00066483430FBF7DAFD0446002C00D0EDE056
:10CCF00000F038FE002815D1022103200AF4ECD7F9
:10CD00005B480F388079012802D100F0B3FE09E0BA
:10CD100000F0EEFE5C484078C007C00F002801D04C
:10CD200001F042FAD2E001F0D1FD0021504811306B
:10CD3000C17300F017FE002815D1022103200AF468
:10CD4000CBD74B480F388079012802D100F092FEF2
:10CD500009E000F0CDFE4C484078C007C00F002825
:10CD600001D001F021FAB1E0687800280BD04048EA
:10CD70000F38C179C079401E3D4B0F3BD871184622
:10CD8000093001F02FFCA1E000BF00BF00BF00BFD1
:10CD900000BF37480F38407901280EDB34480F3880
:10CDA0004079062809DC2878A72804D130480F38B4
:10CDB0000079002801D100F0F1FD2878A42802D0E4
:10CDC0002878A7282BD12A480F384079042806D084
:10CDD000062805D008280ED00C281ED114E000BF6C
:10CDE0002A480068002805D0214A0F3A9079274A3E
:10CDF0001168884712E024480069002803D02248BF
:10CE000001690120884709E01F480069002803D014
:10CE10001D4801690320884700E000BF00BF55E0BE
:10CE2000002013490F390871FF20C870FF211048F6
:10CE300011300175417549E00D481130007DFF2822
:10CE400026D06878002823D10F484078C007C00F4B
:10CE500000281FD001F0A8F91CE00000040D00001C
:10CE6000E42E00200502000048080000A08C00000D
:10CE70006F2E0020B00B0020DC240101680B002085
:10CE80003425010101180000702F0020102F002010
:10CE900000F0A6FE1AE00F48407DFF2812D0687807
:10CEA00000280FD10B48807D00280DD00A4840781B
:10CEB0008007C00F002807D00648C17D183001F058
:10CEC000D1F801E000F06AFE00E000BF00BF0020E2
:10CED0000DB0F0BD802E0020702F0020F8B5064662
:10CEE0000C4617460025002000E0401C0628FCDB0D
:10CEF0003248007E0300FDF716F8060406101C28D1
:10CF0000344001253AE02D480622C169A01CFBF7F8
:10CF1000DCF9002800D1012530E0237E2748224695
:10CF20001A32C169092000F0B1FF002800D00125A4
:10CF300024E0237E214822461A32C169212000F0D4
:10CF4000A5FF002800D0012518E0237E1B482246BB
:10CF50001A32C169162000F099FF002800D001257F
:10CF60000CE0237E154822461A32C169192000F0D0
:10CF70008DFF002800D0012500E000BF00BF104851
:10CF8000807D002817D10D484069002803D00B4848
:10CF9000416920468847002D0DD0084800690028C7
:10CFA00003D0064801690220884701F08BF9217AF5
:10CFB000A01C01F057F80020F8BD0000702F0020E1
:10CFC000802E0020F8B505460C4616461F46042262
:10CFD00021466846FBF728F90098FBF71CF900206A
:10CFE000F8BDF8B506460F46144620460AF462D648
:10CFF0000546012D02D100BF00BF00BF0020F8BDD3
:10D0000030B50446002000E0401C0628FCDB002070
:10D0100030BD0000FEB50D4616461F4630460AF4E8
:10D0200049D601900198002816D1472001F0C0FF91
:10D03000009004233246032108480AF47DD50446B3
:10D040003804000E2070298800988088081A6080B3
:10D0500020460AF4ADD500BF0020FEBD0D470000FC
:10D06000F8B50D461746472001F0A2FF0446287880
:10D07000122802D02878132836D1A06801460C3136
:10D0800000912878122810D1A068C2880189042351
:10D0900016480AF451D506460098408830806878D2
:10D0A000B07030460AF484D511E0A068C2880189C6
:10D0B00006230E48801C0AF43FD506460098408897
:10D0C00070806878307130460AF472D500BFA0686D
:10D0D000002804D0A0680AF41FD40020A06000211A
:10D0E00038460AF4F9D500BF0020F8BD0747000014
:10D0F000FEB505460C4616461F461848006C00282B
:10D100000CD0002000900190029009206946087020
:10D1100001941248016C6846884700BF20780828AF
:10D1200017D008DC01280DD002280ED005280DD01C
:10D1300007280FD10BE00D280AD0122803D013289E
:10D1400008D101E007E006E005E004E003E002E0CA
:10D1500001E000E000BF00BF0020FEBD602E002007
:10D16000FEB506460C4617461D462088154908861A
:10D1700021882804000E020112484830101841810D
:10D180001048006C00280CD0002000900190029004
:10D1900007206946087001940A48016C6846884770
:10D1A00000BF2804000E800007490858002807D057
:10D1B00000212804000E8000034A10584030C1743A
:10D1C0000020FEBD602E0020580B0020FFB587B068
:10D1D0001D4609980AF46ED506900698002878D165
:10D1E000472001F0E5FE0646002105912804000EC7
:10D1F00004900899088805A902F0B7FD0390002063
:10D200000290002101910398002844D16846007DD6
:10D2100016225043316A0818008A03214903084046
:10D220004013002819D16846007D5043316A095CDB
:10D230006846007D16235843326A10184078000271
:10D2400008182549884208D16946097D049802F0EA
:10D25000A2FD0190022002901CE02804010E30463D
:10D2600001F096FE0423009001461C48099A0AF436
:10D2700063D407462804000E38706846007D788025
:10D2800038460AF495D4012109980AF425D50020DE
:10D290000BB0F0BD00BF0298801D83B22946104834
:10D2A000099A0AF449D40446089801882180039910
:10D2B0002171029961800398002804D101A9601DA1
:10D2C000029AFAF7B1FF20460AF472D40020DFE791
:10D2D000FFE70220DCE7000002290000044700000D
:10D2E000140C0000FFB589B00C461E46472001F023
:10D2F0005FFE0746002007903004000E069020884D
:10D3000007A902F032FD05900598002864D168460F
:10D31000007F16225043396A0818008A0321490306
:10D3200008404013002835D16846007F5043396AD1
:10D33000095C6846007F162358433A6A1018407803
:10D34000000208182E49884224D100200290039040
:10D35000208800F095F8054602A800231A4604A983
:10D3600000902846FBF7A0FA6946098A01221203B9
:10D3700011401140080B2146FEF75AFBC0B2059040
:10D380000598002805D1E2886846017F069802F0DA
:10D3900091FD00BF059800281ED13004010E3846CB
:10D3A00001F0F6FD0390A088801D83B215480B9A0A
:10D3B00003990AF4C1D30546A288A11DA81DFAF756
:10D3C00033FF069828706846007F6880A088A88090
:10D3D00028460AF4EDD300BF042331460A480B9ACD
:10D3E0000AF4AAD308902188089801800599089822
:10D3F000817008980AF4DCD300200DB0F0BD000065
:10D40000022900000A470000160C000070B588B021
:10D4100005462C462046FBF74DFA064625E001A9B5
:10D420002046FBF72FFA0020034604AA03A9009028
:10D4300001A8FBF745FA6846008A1049884206D1E0
:10D440006846007B022802D1204608B070BD6846BD
:10D45000008A0A49FF39884204D16846007B0228C5
:10D4600000D108E0601C84B200BFB088A04202DC9A
:10D47000F088A042D3DA00BF0020E6E702290000CE
:10D4800070B588B005462C462046FBF713FA0646D1
:10D4900017E001A92046FBF7F5F90020034604AA8E
:10D4A00003A9009001A8FBF70BFA6846008A094916
:10D4B000884203D1601C80B208B070BD601E84B287
:10D4C00000BFB088A04202DCF088A042E1DA002070
:10D4D000F2E700000328000030B587B004460D468F
:10D4E0000E48844204D101210420FCF715FA09E01A
:10D4F0000B48844204D101210820FCF70DFA01E019
:10D5000007B030BD01A8FBF7ABFF019501200290E9
:10D5100001A92046FBF720FF00BFF1E7000801400A
:10D52000000C014010B50446022C05D1A0200B4987
:10D530000870802048700EE0032C01D0042C05D127
:10D54000E020064908700020487004E0A02003494C
:10D5500008700020487000F089F810BDD006002047
:10D5600010B520202949486001202949C8630520B9
:10D570002849886100202649C8630B202449803946
:10D58000086100F073F8244821498031086323487A
:10D590004863234888632348C86323481C49C03133
:10D5A000086022484860224888602248C8602248B3
:10D5B000086122484861224888612248086322485D
:10D5C000224948602248C86022480861124808621F
:10D5D00021484862124888621248C86212480863AB
:10D5E000124848631D4888631D48C8631D48174991
:10D5F00040310860104848601B4888601248086342
:10D6000013481030886302F087FA10BD0010014003
:10D61000C0270240402502400259F800025B850005
:10D62000025A8000025D8500025F80500200087887
:10D63000020A0800026EAC500259FC000200C80049
:10D640001270131402700314026E2800C0280240E6
:10D65000025D0500125B0500025B8400020A060001
:10D66000026E2C5002C3BF001200AC001B48007DAC
:10D67000FF2809D11948407DFF2805D11848407876
:10D68000C007C00F002810D01648007816498860DF
:10D6900014484078C86115481549086115488862E2
:10D6A000124813494031086017E0104810381049FB
:10D6B000086111484861114888610E481038886235
:10D6C0000D48C8620E4808630848103808494031C0
:10D6D00008600C484860094888607047802E002028
:10D6E000702F0020D006002000270240127E02008A
:10D6F00000280240127E030002C2A00012C70000F0
:10D7000012C7800002C2E000FCF714FA1348144963
:10D710000863FDF7DDFF13A0FCF7B4FB1CA0FCF7CA
:10D72000B1FB25A127A0FCF7ADFB2C4801682CA07C
:10D73000FCF7A8FB31A134A0FCF7A4FB3BA0FCF74D
:10D74000A1FBFDF797FFFDF743F9FBF713F9FBF793
:10D75000FFF803F021F900BFFEE700000080008120
:10D76000007000400A3D3D3D3D3D3D3D3D3D3D3D60
:10D770003D3D3D3D3D3D3D3D3D3D3D3D3D3D3D3DD9
:10D780003D3D3D3D3D3D3D3D3D3D3D3D3D0A000076
:10D79000204E333257423033312046726565525441
:10D7A0004F53202B2055415254202B204C454420D0
:10D7B00064656D6F0A00000056312E30302E303116
:10D7C00000000000204669726D7761726520766501
:10D7D0007273696F6E2025730A000000000000203C
:10D7E0002053797374656D436F7265436C6F636B1F
:10D7F000203D20256C7520487A0A000043414949A4
:10D80000432D4D434D00000020424C4520656E6184
:10D81000626C65642C206164766572746973696EEC
:10D820006720617320222573220A00003D3D3D3DA3
:10D830003D3D3D3D3D3D3D3D3D3D3D3D3D3D3D3D18
:10D840003D3D3D3D3D3D3D3D3D3D3D3D3D3D3D3D08
:10D850003D3D3D3D0A000000F8B505460C46164624
:10D860001F4620780A2815DA207880000A490858CF
:10D870000A4988420ED12078800009490858217849
:10D880008900054A50502178064BC8180321626868
:10D890000AF414D40020F8BDEC2F0020D7040101B5
:10D8A00014300020070F000010B50120C002FBF764
:10D8B000FBFC002806D00120C002FBF7EFFC022091
:10D8C0000A49087001200003FBF7EEFC002805D090
:10D8D00001200003FBF7E2FCFBF718FF0448006897
:10D8E000002802D002480068804710BD8000002058
:10D8F000B80D002000BFEFF3088000BF04480068A7
:10D90000002802D0024800688047FBF7FFFE0000B5
:10D91000B40D00201CB500200090019001200003F0
:10D920000090002168460171082141710121817137
:10D93000FBF7CEFC1CBD00000146094800780A2810
:10D940000CDA0748007882000548001D8150001F4E
:10D950000078401C024A1070012070470020FCE74C
:10D96000E02D002010B500240A48C0790A49097842
:10D9700088420CDA0749C9798A000749091D885885
:10D9800080470448C079401C0249C87101242046E0
:10D9900010BD0000602E0020E02D002010B51D48B5
:10D9A00000790300FCF7BFFA08050C162524282C83
:10D9B0002F3218488079052801D0FDF7A7FA26E014
:10D9C00014488079022802D1FDF786FD01E0FDF7B9
:10D9D000CFFC1CE01048407B002803D10E48C079E2
:10D9E000002802D0FDF778FD01E0FDF705FD0EE00F
:10D9F00000BFFDF771FD0AE006200649087106E048
:10DA0000FDF7AEFD03E0FDF705FB00E000BF00BF42
:10DA100010BD0000602E0020502F002010B50446DD
:10DA2000002C04D0602221461148FAF7FDFB104873
:10DA30002030C0781C2808DD0D484030407B00288D
:10DA400003D11C210A482030C17009484030C078F9
:10DA50001F2803DD1F2106484030C17004484030B4
:10DA6000007BE22803DDE22101484030017310BD54
:10DA7000102F002010B51C480079072803D1012081
:10DA80001949887110BD18488079002804D00128F0
:10DA900006D0052823D104E00120134988711FE036
:10DAA00000BF1248807B002803D002200E498871F5
:10DAB00012E00E48007D002803D003200A49887137
:10DAC0000AE00A48807E002803D0042006498871B5
:10DAD00002E0052004498871FDF718FA00E000BF54
:10DAE00000BF00BFCEE70000602E0020502F0020B6
:10DAF00010B50D4880790300FCF715FA0604050BF4
:10DB00000C0D090A00BF05200749887109E008E0EB
:10DB100000BF00BF00BF052003498871FDF720FD4D
:10DB200000BF00BF10BD0000602E002010B50B48E4
:10DB3000407DFF2810D10223032207216D204001E0
:10DB400009F4FAD70446A22020700548C078607016
:10DB500020460AF42DD000BF10BD0000802E00200A
:10DB6000E42E002010B50B48007DFF2810D10223C1
:10DB7000032207216D20400109F4DED70446A120CD
:10DB800020700548C078607020460AF411D000BFAC
:10DB900010BD0000802E0020E42E002010B50E489D
:10DBA000407DFF2816D00223032207210B4809F4E9
:10DBB000C3D70446A72020700748407D607000202E
:10DBC000054920394871FF2103484175204609F471
:10DBD000EFD700BF10BD0000802E0020A30D000075
:10DBE00010B50C48007DFF2813D002230322072123
:10DBF000094809F4A1D70446A72020700548007DF4
:10DC000060700020034920394871204609F4D0D7BC
:10DC100000BF10BD802E0020A30D000010B50948E4
:10DC2000807800020146083102230322064809F4E5
:10DC300083D704460120207013206070204609F429
:10DC4000B7D710BD602E0020040E000010B584214F
:10DC50001148FAF710FB2A211048FAF70CFB602153
:10DC60000F48FAF708FB20210E48FAF704FBFF20C3
:10DC70000949C870FF21084820300175417500200E
:10DC800007E0FF2203010449483159188A70411CFA
:10DC9000C8B20328F5DB10BD602E0020E42E002062
:10DCA000102F0020702F00201FB50446002C04D038
:10DCB0002A2221461048FAF7B7FA10A30FCB039394
:10DCC0006B4607C3002009E06946095C0A4A121D39
:10DCD000125C11436A461154411CC8B20628F3DB9A
:10DCE000102269460A48FAF79FFA06220249091DDE
:10DCF0000848FAF799FA1FBDE42E00205019219028
:10DD00001F04D5624FA489AB90D0CF230000000040
:10DD10006F2E0020FC0000200021002009E00301FC
:10DD2000064A9A189278FF2A01D04A1CD1B2421CA6
:10DD3000D0B20328F3DB084670470000A82E00206D
:10DD4000F8B507460D46284628214843831C032280
:10DD50000721104809F4F0D60646912030707570FE
:10DD6000002410E0002128206043C019C17128223E
:10DD70006243D11928226243B31CD0182822FAF733
:10DD800053FA601CC4B2AC42ECDB304609F410D745
:10DD9000F8BD0000910D000010B50446032C22D1FF
:10DDA000284880680F2109020843264988602648D0
:10DDB000006A042108432449086200BF2248006A1F
:10DDC000082108400028F9D01F48006A2021084394
:10DDD0001D4908627D20C0001C4908603D200001EB
:10DDE0001B4908602DE01848006A012108431649C4
:10DDF000086200BF1448006A022108400028F9D0D8
:10DE00001148006A202188430F490862002C0ED077
:10DE1000012C02D0022C09D103E00E480B49086006
:10DE20000AE00C4886300949086005E000BF7D2003
:10DE3000C0000649086000BF00BFFAF747FD04496B
:10DE4000086010BD00100140001002408C0000204E
:10DE500090000020D103000001460B4800780A28FA
:10DE60000FDA09480078C2000748001D10184B68F7
:10DE70000A680CC004480078401C034A1070012056
:10DE800070470020FCE700000C2E0020FFB581B099
:10DE9000074614461D461EE02078401CA84201DCBF
:10DEA000032D00DA19E02078401EC6B2641C2078E9
:10DEB0000090641C0098B84209D13246204602996D
:10DEC000FAF703FA002802D1012005B0F0BDA41929
:10DED000B01C281AC5B2002DDED100BF0020F4E727
:10DEE00010B5044600F05EF8FFF7B0FE2249206846
:10DEF00008646068486461891F484030C187207A9F
:10DF0000032804DC217A1C486030417703E00021BB
:10DF100019486030417700BF01212020FBF7ECFC5D
:10DF2000164A1749042000F0B1FF16481649086048
:10DF30000A4613494031052000F0A8FF134A14494E
:10DF4000072000F0A3FF1348134908600A46104950
:10DF50004031082000F09AFF104A1149092000F0D2
:10DF600095FF00BFFBF7E2FA00F0D0F9002001F0C6
:10DF70008FF8FDF7EDF910BD602E0020000700209E
:10DF800080800100551E010140070020800700200D
:10DF900000DB010001080020C0070020400D002028
:10DFA000C0610200F8B5234C234D2449A868C8621B
:10DFB00023480863E86A8862E86B4863A86B886353
:10DFC0007C22294640312046FAF72EF90020606075
:10DFD000E06060621B48A06200206064A064E064AE
:10DFE00020661948A0661948206200201849087068
:10DFF0000320184908700A20FBF7E4FA1A20FBF7FF
:10E00000E1FA0820FBF7DEFAE868461E3788124876
:10E01000874202D01149E8680860286E461E37889A
:10E020000D48874202D00E49286E0860FFF772FC47
:10E03000F8BD0000C009002000800001C0000020E1
:10E04000F5D800018D0D0020C1030101A9D8000100
:10E05000C6000020D8000020FEE70000B40D00201C
:10E06000B80D002070B506460D464A48407DFF2891
:10E0700013D1FFF75BFD4748C575062231461830BE
:10E08000FAF7D2F8012143488175434840780221CC
:10E090008843801C4049487070BD3F48C0680028D4
:10E0A00005D03D480321C2683C480AF407D03A2312
:10E0B000032207213A4809F43FD50446A4202070E2
:10E0C0003448407D6070334860300078002807D0C5
:10E0D0000120A0700021A1802E486030017003E073
:10E0E0000020A0700021A1800121E17019214901C7
:10E0F000E18021812B48018CE181418C2182818C3E
:10E100006182C18CA1820021E182FF214131218302
:10E11000214840784007C00F002815D0E07804213E
:10E120000843E070192149016181A1811D48018CDA
:10E13000E184418C2185818C6185C18CA185002180
:10E14000E185FF21413121863820055506223146DF
:10E1500020463230FAF768F8E078022108400028BB
:10E1600003D00220FFF7DEF90BE0E078042108403D
:10E17000002803D00320FFF7D5F902E00120FFF7C4
:10E18000D1F90C20034920394871204609F410D5F3
:10E1900000BF81E7802E0020702F0020030F0000B9
:10E1A000A10D0000E42E002010B53448007DFF28AA
:10E1B00009D13348407840084000401C304948703D
:10E1C000FFF7D0FC10BD2E484078C007C00F0028D4
:10E1D00000D1F7E72A4840784008400028494870B5
:10E1E00000212648603001703A2303220721254888
:10E1F00009F4A2D40446A42020702048007D607059
:10E200001F480078A0701E4840788006810F217159
:10E210001B484188E18081882181C188E181018991
:10E2200021820121E1700120FFF77CF91448407838
:10E230004007C00F00280BD0E07802210843E070AF
:10E240000F48418861818188A1810320FFF76AF925
:10E250000B4840780007C00F002803D0E0780C215D
:10E260000843E0700820054920394871002103481F
:10E270008175204609F49CD400BFA3E7802E0020BE
:10E28000702F0020A10D000010B50C48407DFF2824
:10E2900013D0022303220721094809F44DD4044670
:10E2A000A52020700548407D60700D20034920396D
:10E2B0004871204609F47CD400BF10BD802E002098
:10E2C000A20D000010B50F48007DFF2818D00D48A2
:10E2D00020384079092813D00223032207210A4855
:10E2E00009F42AD40446A52020700648007D6070F9
:10E2F0000920044920394871204609F459D400BF47
:10E3000010BD0000802E0020A20D000010B50449B1
:10E31000032009F425D50021032009F4DDD410BD24
:10E320003C26010170B504466088A188491C484319
:10E330001921C901884215DC6088062812DB608833
:10E34000218888420EDBE0887D21C900884209DCF3
:10E350006088A188491C484341004018E188C900F1
:10E36000884201DD002070BD0E4880780002014621
:10E3700008310E2303220C4809F4DED30546092098
:10E380002870208868806088A880A088E880E0885D
:10E39000288100206881401EA881284609F408D4FD
:10E3A0000120E0E7602E00200E0E000070B5CAB01C
:10E3B0000446FF2129316846F9F75DFF2448856945
:10E3C000407C002801D14AB070BD00F045F8694694
:10E3D000887089781E48807C814210DA684680788F
:10E3E0003A21484306463246291D01A8F9F71CFF89
:10E3F00068468078401CC1B2684681700CE068466F
:10E400008078401E3A2148430646324629463E312E
:10E4100001A8F9F709FF00BF69468978491E3A2229
:10E42000514301AA88183A222146F9F7FDFE09480E
:10E430006946088006498869FBF702FA0449FF2209
:10E44000273288696946FBF735FA00BFBBE7000051
:10E45000CC2F00203412000070B5002400260A489A
:10E4600085692E88AC780948864209D10648807CA7
:10E47000A04206DA002404498869FBF7E1F900E0CC
:10E480000024204670BD0000CC2F00203412000074
:10E490000EB500200290FBF7F1F9FFF7DDFF0290C7
:10E4A0000E48C06900280CD0002000900190012087
:10E4B0006946087002A801900848C1696846884703
:10E4C00000BF6846007A002803D001200349087085
:10E4D00002E00020014908700EBD0000CC2F002092
:10E4E000F8B504460D463A26054887693A20604348
:10E4F0003A1D811832462846F9F796FEF8BD00000D
:10E50000CC2F002030B58FB0044600253C21684652
:10E51000F9F7B1FEFFF7A0FF0546691EC8B26946CC
:10E52000FFF7DEFF08A8807CA07106220CA903314A
:10E530002046F9F779FE0FB030BD30B58FB00446F4
:10E5400000253C216846F9F796FEFFF785FF054652
:10E55000691EC8B26946FFF7C3FF06A80230807D76
:10E56000A07106220AA902312046F9F75DFE0FB01C
:10E5700030BD000030B58FB0044600253C21684610
:10E58000F9F779FEFFF768FF0546691EC8B26946CC
:10E59000FFF7A6FF06220AA902312046F9F744FE3A
:10E5A00006A80230807DA071102206A90231204603
:10E5B0000830F9F739FE0948C078012806D1102241
:10E5C000074920461830F9F72FFE04E010212046B5
:10E5D0001830F9F750FE0FB030BD0000E42E0020D7
:10E5E0006F2E0020F0B58FB006460D46FFF734FFC2
:10E5F0000746002D25DDBD4223DC18230322072119
:10E60000114809F499D20446172020700120607047
:10E6100006223146A01CF9F707FE3C216846F9F7AF
:10E620002AFE691EC8B26946FFF75AFF102206A9E2
:10E63000023120460830F9F7F7FD204609F4B8D238
:10E6400000BF0FB0F0BD0000140D0000F0B58FB09A
:10E6500007460D463C216846F9F70DFEFFF7FCFE24
:10E660000646012D0AD11448C671C179C079401EF1
:10E67000114BD8713846FFF7B5FF1BE0344616E062
:10E68000611EC8B26946FFF72BFF06220AA90231B4
:10E690003846F9F71AFE002807D1102206A90231E0
:10E6A00005481F30F9F7C0FD03E0601EC4B2002C1E
:10E6B000E6DC00BF0FB0F0BD602E00200F48C08F19
:10E6C0000A281ADD0E48C0690121090708430C49D0
:10E6D000C8610B4840304068012108430849403177
:10E6E0004860084808490860032048600348C08F14
:10E6F000886006480860064808607047A02E002021
:10E70000001002405555000000300040AAAA000049
:10E71000CCCC00001CB500BF23480068012149048F
:10E7200008400028F8D02149487FFFF735FB1E48F4
:10E73000406A1D48406A012108431B494862084657
:10E74000406A400840004862FFF7B8FF68461CF482
:10E7500085D71749009808601448407F03281AD0CD
:10E7600000F0D6F81048006BFF21090288430E49DB
:10E7700008630846006B3F21490208430A490863C1
:10E780000846006B01210843074908630122032161
:10E79000084809F493D400210120FAF77BFF0021F7
:10E7A0000A20FAF777FF1CBD00100240C02E00209F
:10E7B000BC0D0020010F0000F0B58FB005460E46DD
:10E7C00017460DA81CF44AD700200B900C9000BFF0
:10E7D0003849886A00BF0B9000BFC86A81B20C91AB
:10E7E0000D990B98401A000100090121C9068842C1
:10E7F00006D90B990D98401A00010009404204E027
:10E800000D990B98401A000100090446402C03DCC6
:10E810002948408800283FD12848FFF7C7FDFF203E
:10E82000F53025494880282101A8F9F724FD062262
:10E8300022492A3101A8F9F7F7FC20481A30807DD7
:10E840006946887210221D491A3103A8F9F7ECFCB9
:10E850001B48C078012805D110221A4907A8F9F7EA
:10E86000E3FC04E000200790089009900A90012141
:10E8700014481130C1736846807A002807D10F48C8
:10E880002030807C002802D001A8FFF759FA01212E
:10E890000C487130017009E007484088401E064965
:10E8A000488014220321084809F408D400200FB03E
:10E8B000F0BD0000C0800240CC2F0020902F00202F
:10E8C000E42E00206F2E0020040F00000348007883
:10E8D000002801D0012070470020FCE7CC2F002049
:10E8E0000148007970470000CC2F002010B5044685
:10E8F0001C2221460548F9F797FC0448001F407C7C
:10E90000002801D0FFF7C4FD10BD0000D02F00206B
:10E91000054801680068401C034A1060002901D1C5
:10E92000002070470120FCE7401B002006480068DB
:10E93000002806D004480068401E034908600120F2
:10E9400070470020FCE70000401B0020FFB581B0AD
:10E9500004460E4617460A9D16482018002802D085
:10E96000012813D109E03A4631462046049BFDF7C1
:10E9700027F82870002005B0F0BD3A463146204601
:10E98000049BFEF769FF28700020F4E70A488442E0
:10E9900003DBF1200001844202DD01202870EAE758
:10E9A0000549611AC8B2FCF7E5FF0020287000BFD6
:10E9B000E1E70000FBF0FFFF070F000010B50C4877
:10E9C000006800030B49096844182046FAF738FF2D
:10E9D000002801D0052010BD01221203064920465F
:10E9E000FAF768FF002801D00520F4E70020F2E7DD
:10E9F000582900204429002088920020F7B582B0D1
:10EA00000C4604980C2807D00023012210210298FC
:10EA100000F0BEF905B0F0BD204600F0ADF90546A6
:10EA2000201D00F0A9F901902046083000F0A4F95B
:10EA30000090FCF763FC06462248864202D141273B
:10EA4000BF040CE041208004864201D11D4F06E046
:10EA5000002302221021029800F09AF9DAE7042D2F
:10EA600003D30720C003854206D9002303221021C7
:10EA7000029800F08DF9CDE713480078002804D102
:10EA8000FAF7FCFE01201049087001200F490870B8
:10EA90000F4807600F4805600F49019808600F494B
:10EAA0000098086000200E4908600E4908600E4971
:10EAB000086000231A461021029800F069F900BF8F
:10EAC000A8E7000000800001602900204029002004
:10EAD00044290020482900204C29002050290020EA
:10EAE00054290020582900205C290020F7B584B063
:10EAF0000E46174641480078002807D1002302221D
:10EB00001121049800F044F907B0F0BD042F07D29A
:10EB10003B48012211210368049800F039F9F3E71A
:10EB2000304600F029F90390301D02903C1F344913
:10EB300003980968884207D03148022211210368EE
:10EB4000049800F025F9DFE72D48006800192D49E9
:10EB50000968884207D92A480322112103680498CA
:10EB600000F016F9D0E744E02748006801210903C6
:10EB70000D1AA54200D925462449234A126888184F
:10EB80002A460299F9F750FB1F48006840191E49B0
:10EB90000860029840190290641B194800684019E7
:10EBA00017490860184800680121090388421FD1ED
:10EBB000FFF704FF01900198002809D0104803686E
:10EBC0001121019A049800F0E3F8FCF785FB9BE71C
:10EBD0000F480068401C0E49086000200A49086080
:10EBE0000748002211210368049800F0D1F800BF03
:10EBF00000BF002CB8D100BF86E7000040290020EC
:10EC000054290020482900205C29002088920020F7
:10EC100058290020F7B582B00E4617464C480078B8
:10EC2000002807D1002302221221029800F0B0F838
:10EC300005B0F0BD042F07D0464801221221036819
:10EC4000029800F0A5F8F3E7304600F095F8054685
:10EC50004048006840490968884207D03D48022280
:10EC600012210368029800F093F8E1E73B4800683E
:10EC7000002832D03A48006800033A490968401831
:10EC8000019036480068C01C80088000009008E0B1
:10EC9000FF21324802680068401C304B186032483F
:10ECA00081542E48016800988142F1D30198FAF707
:10ECB000C7FD002806D12C49009A0198FAF7FAFD01
:10ECC000002809D02348052212210368029800F089
:10ECD0005FF8FCF701FBABE700BF1F480168214864
:10ECE0000068FCF725FE0446AC4203D11F480068CB
:10ECF000844209D01748042212210368029800F0C8
:10ED000047F8FCF7E9FA93E700F05EF8002809D02D
:10ED10001048052212210368029800F039F8FCF728
:10ED2000DBFA85E70C48002212210368029800F004
:10ED30002FF8C82001F0E2FC00BFBFF34F8F0C4852
:10ED40000C49C860BFF34F8F00BF00BFFEE7000053
:10ED50004029002054290020482900205C29002057
:10ED60005829002044290020889200204C290020A6
:10ED70000400FA0500ED00E0014608784A78120226
:10ED800010438A7812041043CA7812061043704761
:10ED9000FEB505460E4617461C4668460670477087
:10EDA00084702004010E6846C1702002010E68467E
:10EDB0000171200E6946487106236A4629461F20C4
:10EDC000FBF7ACFFFEBD000010B58AB02422284935
:10EDD00001A8F9F729FA27490198884206D120218C
:10EDE0002348FCF7A5FD0999884203D0242101A8F6
:10EDF000F9F741FA1F4801901F4800681F498842EF
:10EE000001D1012000E0022002901B4800681B494C
:10EE1000884201D103A800E006A80446184800680B
:10EE2000206018480068606017480068A0602021D2
:10EE300001A8FCF77DFD09900D48FAF701FD0028B7
:10EE400002D005200AB010BD242201A90848FAF713
:10EE500031FD002801D00520F4E72422044901A84F
:10EE6000F9F733FA002801D00520EBE70020E9E7A5
:10EE70000040000111C011CA442900200080000197
:10EE8000482900204C2900205029002030B51028A6
:10EE900000D330BD114B84001B591B0B1B038C038B
:10EEA000240D23430D4C85006351234684001B59D8
:10EEB0000B4C234094092403094DED432C4023437C
:10EEC000064C85006351054B183B5B690124844067
:10EED0002343024C183C636100BFDAE7182002406C
:10EEE000FF0FC0FFF3B583B005460026688800F029
:10EEF00035F902900298002800D14026002E10D14A
:10EF000000240BE01420604320494018408A69889F
:10EF1000884201D1422603E0601CC4B20A2CF1DB16
:10EF200000BF002E2FD1002427E014206043174992
:10EF30004018408AFF281ED12846083000906B7880
:10EF4000AA8814206043401801900298A91D076800
:10EF50000198B8470646002E0CD1698814206043FA
:10EF60000A4A801841821420604311464018018AE1
:10EF70000498018003E0601CC4B20A2CD5DB00BFFA
:10EF80000A2C00D14B26304605B0F0BDC42C002021
:10EF900010B5024613885804400C13880124E4037A
:10EFA0002340DB13002B01D00B02184310BD0000DF
:10EFB00010B50246002000210DE014234B43084CFD
:10EFC0001B195B8A934204D114234B431B19D86845
:10EFD00003E04B1CD9B20A29EFDB00BF10BD0000D3
:10EFE000C42C002030B50146FF230804040EC9B22A
:10EFF00000220DE014205043084D4019008A884239
:10F0000004D1142050434019438A03E0501CC2B27B
:10F010000A2AEFDB00BF2002184330BDC42C0020B9
:10F0200001460B4800780A280FDA09480078C20028
:10F030000748001D10184B680A680CC00448007887
:10F04000401C034A1070012070470020FCE70000BC
:10F050008C2D002030B50146FF230804040EC9B2F0
:10F0600000220DE014205043084D4019408A884288
:10F0700004D1142050434019038A03E0501CC2B24B
:10F080000A2AEFDB00BF2002184330BDC42C002049
:10F0900070B50546002D01D12E490870002456E0B8
:10F0A000002D04D0012D32D0022D4CD117E0204686
:10F0B000093014216143284A8918088214216143C8
:10F0C0008918087C08F466D614226243224BD118B2
:10F0D00014226243D218107C08F442D634E0142182
:10F0E00061431D4A8918488A00F038F80646002E08
:10F0F00005D014226243184BD01871688847142138
:10F100006143154A8918087C08F468D600BF0021BD
:10F1100014206043104A8018C160FF21142060430E
:10F120008018418200211420604311501420604354
:10F1300080184160142060438018018114206043CE
:10F140008018418100E000BF00BF601CC4B20A2CDF
:10F15000A6DB70BD8C2D0020C42C0020F8B5054620
:10F160000026EFB200240CE0E1000948405AB84202
:10F1700005D1E20006495118486880470646601CE0
:10F18000C4B20348001F0078A042EDDC3046F8BD51
:10F19000902D0020F8B50446FBF77CFC0546F42DC5
:10F1A00000D9F425072D00DCF8BDE81F86B213E076
:10F1B0002046F9F76BF887B2B74200DD37460948B9
:10F1C00001780078401C074B18703B46224602200D
:10F1D000FBF7A4FDE41900BF20780028E8D100BFA8
:10F1E000E2E70000CD28002070B502460B460F482C
:10F1F000002117E0555C2D02684000240EE0012537
:10F20000ED030540002D04D04500094E7540ADB218
:10F2100001E045042D0C2846651CECB2082CEEDB01
:10F220004D1CA9B29942E5DB70BD0000FFFF000054
:10F2300021100000FFB581B0054616461C46012D81
:10F2400006D0102D22D0112D21D0122D27D11FE054
:10F2500001273F2C11DC224631461348F8F7E4FF22
:10F260000020114908551148FCF714FD0E48FCF721
:10F2700007FC07460020FCF70DFDF8B200900123C3
:10F280006A4603200299FBF749FD09E000BF00BF71
:10F290002346324628460299FCF734F800E000BFC6
:10F2A00000BF05B0F0BD00003735002095F100012A
:10F2B00070B505460C46FBF7E7FB002801D1401E60
:10F2C00070BD14480088002806D121462846FBF767
:10F2D00023FC002800D1F3E70E4800880019012123
:10F2E000490288420ED80C490A4A128888182246D8
:10F2F0002946F8F799FF0748008800190549088052
:10F300000020DDE705480088401C044908800020F3
:10F31000C043D5E7CE28002037330020D028002076
:10F32000F8B505460E461748076817480068001DDF
:10F3300001F0D2F8681C002808D1002E06D012482F
:10F340000168091D114801F05EF91AE07C190E48A8
:10F3500000684460BC4207D20B480168091D0C4894
:10F36000006801F035F90CE007480168091D0948FB
:10F37000006801F02DF908480068844201D206486F
:10F380000460F8BDE8280020D4280020543600206E
:10F39000DC280020D82800200429002010B50446CD
:10F3A00001F03EF922480068401C214908602148CC
:10F3B0000068002808D11F4804600846006801283A
:10F3C0000ED100F097F90BE01B480068002807D128
:10F3D00018480068C06AE16A884201D8154804608C
:10F3E00016480068401C15490860084600686064BB
:10F3F0001349E06A0968884202D91149E06A086045
:10F400001422E16A51430F4A8818211D01F0FBF8CC
:10F4100001F014F908480068002807D00548006882
:10F42000C06AE16A884201D201F05CF910BD0000B7
:10F43000E4280020D4280020F02800200029002003
:10F44000EC2800207835002010B516E001F0E8F82F
:10F450000C48C068C468201D01F03EF80A480068E6
:10F46000401E0949086009480068401E07490860B5
:10F4700001F0E4F8204600F061F804480068002834
:10F48000E4D110BD40360020E4280020E028002010
:10F4900070B504460D46206C00280ED0216CE06843
:10F4A0004018E0606168E068884201D32068E0604D
:10F4B0002846226CE168F8F7B7FE70BDF8B504463F
:10F4C0000F46154600200090A66B206C002809D13D
:10F4D000206800282ED1606801F000FF0090002015
:10F4E000606027E0002D0FD13946226CA068F8F744
:10F4F0009BFE216CA0684018A0606168A0688842EB
:10F5000018D32068A06015E03946226CE068F8F74F
:10F510008BFE216CE068401AE0602168E068884258
:10F5200003D2216C6068401AE060022D02D1002EE7
:10F5300000D0761E701CA0630098F8BD10B504467C
:10F54000206B01F08FF8204601F08CF810BD0146C9
:10F550004A6A002A04D00A6B12680723981A00E04E
:10F560000020704730B50B23DB0217484407640FB7
:10F57000002C05D0C01DC008C000134C041B1B1B71
:10F580000246124C22600024104D6C60D0180838DE
:10F59000C008C0000E4C206000240D4D2D686C602A
:10F5A0000B4D2D682C601146441A4C60084C2468A1
:10F5B0000C60084D4C682C60074D4C682C60012491
:10F5C000E407064D2C6030BD683600201429002069
:10F5D0001C2900202429002020290020282900207F
:10F5E00000BFFFF731FF034800680128F9D901F097
:10F5F00079F8F6E77835002010B50446002C09D0DC
:10F60000002060602060E06000231A461946204612
:10F6100001F0E0FA10BDFFB581B006460D46174671
:10F620000A9C002D01D1246000E02760E663256478
:10F630000121204601F08DFA4C210498085505B0AF
:10F64000F0BDFFB581B00F460A9E0C9C039A910055
:10F65000A522206BF8F708FE216B0398401E80005E
:10F66000081800900098C008C0000090009840075B
:10F67000400F002801D1012000E00020002802D125
:10F6800072B600BFFEE7002508E0795D2046343001
:10F690004155785D002800D102E06D1C102DF4D397
:10F6A00000BF002143200155072E00D30626E66245
:10F6B000E66400202065201D00F087FF20461830FA
:10F6C00000F083FF24610720801BA061646200209A
:10F6D0006065002158200155049A0199009800F0B6
:10F6E0000BFA20600B98002801D00B98046005B03D
:10F6F000F0BD000010B5002406E0142161430E4A5D
:10F70000881800F055FF641C072CF6D30B4800F056
:10F710004FFF0B4800F04CFF0A4800F049FF0A4831
:10F7200000F046FF094800F043FF0448084908601C
:10F7300003480849086010BD7835002004360020D1
:10F74000183600202C360020403600205436002089
:10F75000D8280020DC28002010B50146164800E01B
:10F76000006803688B42FBD3024643689B188B42B8
:10F7700004D143684C681B19436001460A464B6834
:10F780009B180468A34211D10C4C03682468A3425F
:10F7900008D04B68046864681B194B6003681B68D9
:10F7A0000B6005E0054B1B680B6001E003680B6014
:10F7B000884200D0016010BD142900201C290020BF
:10F7C00070B5054600F02CFFA86B002801D101247C
:10F7D00000E0002400F032FF204670BD70B5054601
:10F7E00000F01EFFA86BE96B884201D1012400E004
:10F7F000002400F023FF204670BDF7B582B0074615
:10F800000C4600262068002829D020464168496817
:10F8100041600146083142688A4202D14168496824
:10F8200041604168C968019100BF2046416849684C
:10F8300041600146083142688A4202D14168496804
:10F8400041604168CD6824207043C11901222846D7
:10F85000049B00F075FF761C01988542E5D1304687
:10F8600005B0F0BD0B4909680968002901D10121E3
:10F8700000E00021002904D00021C943064A11609C
:10F8800006E004490968C968C868034A416811600C
:10F8900070470000D82800200429002010B500205F
:10F8A0000749086188617D21C90006480068F8F7AA
:10F8B00063FC401E024948610720086110BD00003A
:10F8C00000E000E0000000200246002101E0521CA0
:10F8D000491C1078A528FAD0890888B27047000022
:10F8E00007480068401C002801D1012000E00020EA
:10F8F000002802D172B600BFFEE772B600BFFEE775
:10F900001029002070B5044600F08AFE45200557F6
:10F9100013E0606A002801D1012000E000200028E7
:10F9200008D12046243001F06FFD002803D000F0FC
:10F93000BFFF00E003E0681E45B2002DE9DC00BF18
:10F940000021C9434520015500F078FE00F068FE13
:10F950004420055713E02069002801D1012000E070
:10F96000002000280AD12046103001F04DFD00286B
:10F9700001D000F09DFF681E45B200E001E0002DBF
:10F98000E9DC00BF0021C9434420015500F056FEC8
:10F9900070BD70B505460E4631462846F8F7A2FC04
:10F9A0002846F8F773FC044602E020202855641C22
:10F9B0000F2CFAD300202855281970BDF8B504463D
:10F9C0000020009001F01EF83E480068002801D198
:10F9D000FFF7C8FD3C4800682040002861D1002C9A
:10F9E00015D008346007400F002810D06007400F82
:10F9F0000821081A04196007400F002801D10120CE
:10FA000000E00020002802D172B600BFFEE7002C03
:10FA100047D02E480068844243D82D4E30460568B2
:10FA200001E02E462D686868A04202D228680028AE
:10FA3000F7D124480068854233D030680830009000
:10FA4000286830606868001B102813D92F197807C0
:10FA5000400F002801D1012000E00020002802D141
:10FA600072B600BFFEE76868001B78606C603846BD
:10FA7000FFF772FE154968680968081A134908609B
:10FA80000846006813490968884203D20F48006895
:10FA9000104908600C4968680968084368600020DC
:10FAA000286001F0F5FC00984007400F002801D1C4
:10FAB000012000E00020002802D172B600BFFEE75E
:10FAC0000098F8BD1C2900202829002020290020AA
:10FAD000142900202429002006480068002806D0A8
:10FAE0000449096808465030096D491C0160014805
:10FAF00000687047D4280020001F01231B06036004
:10FB0000001F0160001F034B03601438026020389F
:10FB100070470000E1F800010A4800680A4988427D
:10FB20000ED2084800680949884209D90848006887
:10FB30000849086308480068486308480068886303
:10FB400070470000C006002040317A0090D76A005C
:10FB5000C4060020C0260240C8060020CC060020B3
:10FB6000F8B507460D4616464720FFF721FA0090E4
:10FB700000BF00980069044608E02079B84204D12B
:10FB800060792880A01D306002E02468002CF4D148
:10FB900000BF002C02D1002028803060002C01D052
:10FBA0000020F8BD0A20FCE7F8B50C4616463046A2
:10FBB00008F480D00746002F17D14720FFF7F8F947
:10FBC0000090062332461946094807F4B5D7054682
:10FBD00000988088618840182880A0886880A07973
:10FBE0002871284607F4E4D700BF0020F8BD0000C4
:10FBF000180C0000F7B506460D464720FFF7D8F968
:10FC0000074600BF3869044610E02079B0420CD1A5
:10FC10006079A84208D0214638461030F8F75CFEDB
:10FC2000204607F479D6002402E02468002CECD1A9
:10FC300000BF002C0AD128460830012107F4F6D66F
:10FC40000446214638461030F8F74CFE267165719F
:10FC50002A46A01D0299F8F7E7FA0020FEBD000031
:10FC6000F8B506460F46F56801241EE016206043ED
:10FC7000296A0818008A0321490308404013002814
:10FC800012D116206043296A095C162060432A6A53
:10FC900010184078000208180649884204D1E1B2E1
:10FCA0000022384600F006F9641C287FA042DDDC03
:10FCB000F8BD000002290000F8B506460F46F568B9
:10FCC00001241EE016206043296A0818008A0321D7
:10FCD000490308404013002812D116206043296AC6
:10FCE000095C162060432A6A101840780002081840
:10FCF0000649884204D1E1B20022384600F0DAF821
:10FD0000641C287FA042DDDCF8BD00000229000051
:10FD100070B50446E56808E028461030F8F7E8FDBD
:10FD20000646304607F4F8D500BF00BF2969002910
:10FD300001D1012100E00021084600BF0028EBD0DE
:10FD40000020E060284607F4E7D570BD70B5044692
:10FD50004720FFF72DF905460026A879A04202DDCD
:10FD6000A888001986B2304670BDF8B504460E4624
:10FD70004720FFF71DF905468027A888A04208DC28
:10FD8000A888A9794018A04203DD2879201A30708C
:10FD900000273846F8BD7CB504460D466A4601A9E1
:10FDA0002846FFF7DDFE0098065D30467CBDFFB5B6
:10FDB00087B005461F46109E00200690317801202E
:10FDC0008840401E059038460C21084002213940E9
:10FDD0000843014640312A8A00237068009301924B
:10FDE00003910290337805AAB1680898F8F786FD68
:10FDF0000690069800282ED10121282007F416D657
:10FE00000446304607C862622162E061EC600898EF
:10FE10000088A080207FA071F807C00F002802D0C2
:10FE20000120C00300E00020099908432080288AAF
:10FE3000608047206882284600F054F82046103041
:10FE4000F8F762FD217F206A00F008F8288A002177
:10FE500007F442D700BF06980BB0F0BDF8B50546D1
:10FE60000E460020009001241BE01620604340193C
:10FE7000008A0321490308404013002810D11620AE
:10FE80006043295C1620604340194078000208183E
:10FE90000549884204D1E0B26A460421FFF7AAFE70
:10FEA000641CB442E1DBF8BD022900000048704741
:10FEB000DC1D0101FEB504460D46164601AA02A945
:10FEC0002846FFF74DFE684602890199F8F7ACF91C
:10FED00069460E556A46684601892846FFF78AFE3C
:10FEE000FEBD000070B504464720FFF761F80546E7
:10FEF0000448206009206081284618306060012095
:10FF0000208170BDEC1D0101FFB589B00D46472071
:10FF1000FFF74EF80446A0886988401880B2079021
:10FF2000287804900B9807F4C5D60390039801280D
:10FF300002D102200DB0F0BD0798FDF767FA0890D6
:10FF400006A90898FFF711FF05900598002801D031
:10FF50000220EFE701210B9807F4BED600BF284628
:10FF60000C38A060002020736846007E6073607BC0
:10FF700001AA02A9FFF7F4FDA06806460C3600BFEF
:10FF800001990498085C02210840002822D0B0881A
:10FF9000083083B2A068C28804980002811DC12085
:10FFA000000107F4C9D5074613203870A08871886E
:10FFB0004018B880B088F880B288B11D3846083043
:10FFC000F8F732F9384607F4F3D501210B9807F416
:10FFD00083D602E0A06807F49FD40120AAE7FFB50A
:10FFE00089B00D464720FEF7E3FF0446A0886988E4
:10FFF000401880B20790287806900B9807F45AD6DC
:020000040101F8
:1000000003900398012802D102200DB0F0BD07989B
:10001000FDF7FCF9089005A90898FFF7A6FE0490E3
:100020000498002801D00220EFE700BF28460C38D2
:10003000A060069820736846007D6073607B01AA0B
:1000400002A9FFF78DFDA06806460C3600BF019996
:100050000698085CC007C00F002806D101990698D1
:10006000085C02210840002822D0B088083083B202
:10007000A068C28806980002811DC120000107F413
:100080005BD5074612203870A08871884018B88068
:10009000B088F880B288B11D38460830F8F7C4F847
:1000A000384607F485D501210B9807F415D602E0F0
:1000B000A06807F431D40120A7E7F8B506460C463E
:1000C00017464720FEF774FF0546AA886388D218B2
:1000D00090B2A188A31D0022FBF75CFA0020F8BDB6
:1000E000F8B50C461646304607F4E4D50746012F0E
:1000F00035D1A07900281BD1A088801D83B220783B
:100100000002811D3246174807F416D50546A0782F
:10011000FFF71CFE288000202871A0886880A28834
:10012000E11D681DF8F780F8284607F441D512E074
:1001300020780002811D062332460A4807F4FCD4C9
:100140000546A078FFF702FE288080202871284607
:1001500007F42ED500BF0021304607F4BDD500209E
:10016000F8BD0000140C000070B5D2B000240025CA
:1001700000BFEFF310800646FF21453101A8F8F7D4
:100180007AF801AC01349822074901A8F8F74CF835
:100190000120F9F7D6FEA04705463046F9F7D1FE13
:1001A000284652B070BD0000C0160101F8B500200D
:1001B00001214907086007F415D4594802885948B5
:1001C0000168002007F49AD457480288574801680C
:1001D000012007F493D45648008882B2554801683C
:1001E000022007F48BD45448008882B25348016837
:1001F000032007F483D45248406AF0210843504951
:10020000486250481AF46CD40020502102220B4658
:1002100004060D042C4315022C431C434A4D2C604C
:1002200000BF0F200821002203040C0223431343C4
:100230002C46636100BF00206A210822582304066F
:100240000D042C4315022C431C433F4DAC6000BFF2
:100250000520422102020A432B46DA6000BF062035
:1002600005210A460F2304060D042C4315022C43D6
:100270001C43354DAC6100BF03200F210A46030625
:100280000C04234313432C46E36100BF00200146C6
:1002900002460323012405464027009786074F079F
:1002A0003E4317063E439F053E4327053E432F042A
:1002B0003E43009F3E43244F403FBE6300BFFDF7D7
:1002C0004FF961070968C8B2F8F724FB1F480078A6
:1002D000002807D000201AF449D704462146002000
:1002E000F8F71EFB012149070968C8B2F8F71EFBA1
:1002F000F8F722FB012149070968C8B21AF4C2D4F1
:10030000012149070968C8B21AF4CAD40121490772
:100310000968C8B21AF486D6012041070860F8BD02
:100320001C010020180100202401002020010020D1
:1003300034010020300100202C0100202801002081
:1003400040250240740200208080024062000020AC
:10035000F0B589B007460C462068C01920602068B7
:100360004508002620686919401A20601248006874
:10037000F8F7B0F80022114B05910490F8F732F825
:10038000079106903E203946F8F7DCFA4019714192
:1003900001910090F8F7ACF803910290079B069A40
:1003A000F7F7B8FF05910490F8F7B0F805460E4648
:1003B0002846314609B0F0BD9000002000408F4033
:1003C00010B500BF1348C069044602202040002831
:1003D0001ED0012041000F4A116200BF00F024F836
:1003E000FDF7BEF80C480078410040180B49401852
:1003F00040780B49C8610848007841004018074917
:100400004018807806494031C860002005490870CE
:1004100010BD000000800240D2060020881A0101B1
:100420004025024080000020F8B500BF2548806BC1
:10043000009008201AF43ED701201AF449D7224927
:100440000098FFF785FF05460E46204A0023284600
:100450003146F7F7A7FE044620461C49F8F772FA22
:10046000281A1B49081A87B201202146C2070A43ED
:10047000144B40335A6000BF38461946086000BF2D
:1004800001201049096B08229143C20011430D4A13
:10049000116300BF002011468969072212079143AA
:1004A00002071143074A916100BF01201146896983
:1004B00081430143916100BF00BF1146086200BF44
:1004C000F8BD000000800240B80200207102000068
:1004D000700200007047704701460A694B688868DF
:1004E00098608B68486858605068884201D1886875
:1004F0005060002008611068401E1060106870474E
:100500000148006870470000E4280020F7B5054660
:1005100016460024072700F075FA1F49019809685C
:10052000884234D300BF7F1E14227A431B4BD1185C
:100530002422624350190122FFF75FF90419002FAA
:10054000F1D1242161434819022215490968FFF7B6
:1005500054F90419242161434819022211490968F8
:10056000FFF74BF9041924216143481904220E496D
:10057000FFF743F9041924216143481903220B4969
:10058000FFF73BF90419002E01D00020306000F085
:100590007FFF2046FEBD0000E428002078350020C3
:1005A000D8280020DC2800204036002054360020C7
:1005B0000146083141600021C9438160014608318C
:1005C000C160016100210160704700210161704735
:1005D00010B502460B685C1C002C01D1106907E0C5
:1005E0001046083000E04068446824689C42FAD90C
:1005F00044684C604C68A160886041600A6114687E
:10060000641C146010BD42684A6093688B609368F4
:1006100059609160086103685B1C036070470000CB
:1006200072B605480068401C03490860BFF34F8F4D
:10063000BFF36F8F70470000102900200848006842
:10064000002802D172B600BFFEE705480068401ED0
:100650000349086008460068002800D162B6704768
:100660001029002070B506463546002E35D0083DCD
:100670002C461A49606809680840002801D001200A
:1006800000E00020002802D172B600BFFEE720681B
:10069000002801D1012000E00020002802D172B61C
:1006A00000BFFEE70D49606809680840002814D0C3
:1006B0002068002811D10949606809688843606092
:1006C00000F0A0F90649606809684018044908600C
:1006D0002046FFF741F800F0DBFE70BD282900201E
:1006E000202900200120000703494860BFF34F8FF5
:1006F000BFF36F8F7047000000ED00E070B5044657
:100700000025002C14D00D480068002801D10120DC
:1007100000E00020002802D172B600BFFEE700F022
:1007200071F900212046FEF7FBFD00F0B1FE054601
:10073000002D01D1FFF7D6FF70BD00000C2900206D
:10074000FFB581B007460C461E46002F02D11C485B
:10075000006800E038460546256028463430606071
:10076000E86A2061286BE061686CA060E86C6061F9
:100770000020A061052E13D011480068854202D1E7
:100780000020207310E02673032E0DD100F03AF9FB
:10079000A86A002801D00220207300F079FE03E04F
:1007A0002846FBF7A1FB20730398002804D0286B90
:1007B000FFF78AF8208401E00020208405B0F0BD16
:1007C000D428002003490968016003490968416091
:1007D00070470000FC280020E82800207FB505466F
:1007E000002028702D48006803902C4909682422B5
:1007F00051430846FFF7E2F80446002C4DD0002292
:1008000020460399FFF782FE0390002002903DE00E
:100810002421029848430019007B0300F9F783FB69
:10082000050406080A0C0E00582609E0522607E0C7
:10083000422605E0532603E0442601E0002600BFDF
:1008400000BF242202985043001941682846FFF750
:10085000A0F8054624210298484300198068242204
:10086000029951430919098C009101900298504353
:10087000001932460AA103692846F9F713FB2846F6
:10088000F7F704FD45190298401C0290039902985D
:100890008842BDD32046FFF7E5FE7FBDE428002057
:1008A0000925630925750925750925750D0A0000B7
:1008B0000120014908607047F828002070B50446FF
:1008C0000D46002C02D172B600BFFEE70548016854
:1008D00018312046FFF77CFE01212846FEF720FD57
:1008E00070BD0000D4280020FEB506460F463446F1
:1008F00001200090002E48D0206D002802D172B651
:1009000000BFFEE7E06CB84201D23D4600E0E56C76
:10091000E06AA84239D0206D012836D11B48006812
:10092000844201D0012000E00020002802D172B6EC
:1009300000BFFEE7E06A0190E562A069C00FC00752
:10094000002802D10720401BA06161691422019890
:1009500050430F4A8018814201D1012000E000205D
:10096000002812D0201DFFF7B7FD0A49E06A096888
:10097000884202D90749E06A08601422E16A5143BB
:10098000034A8818211DFFF73EFEFEBDD428002033
:1009900078350020EC2800201CB5134800210B46B8
:1009A00080220091019011A1124800F0B3FB04468F
:1009B000012C0DD172B60020C0430F490860012000
:1009C0000E49086000200E49086000F06FF80AE048
:1009D000601C002801D0012000E00020002802D186
:1009E00072B600BFFEE71CBD0829002049444C45F3
:1009F00000000000E1F5000104290020F02800209B
:100A0000E828002002480068401C0149086070473F
:100A10000C2900201A480068002803D00120194939
:100A200008602CE00020174908601748016805E0BD
:100A3000002902D172B600BFFEE7491E14204843C8
:100A4000124A1058002801D1012000E0002000289F
:100A5000EED114224A430D4BD018426852684260CE
:100A6000024608324368934202D1426852684260AB
:100A70004268D268064B1A600348016000BF7047A5
:100A80000C290020F8280020EC28002078350020D0
:100A9000D428002001480068704700002029002069
:100AA00001480068704700002429002010B50B4859
:100AB000006AFF2109040843084908620846006AE1
:100AC000FF210906084305490862FEF7E7FE0020FA
:100AD00003490860F7F706FB002010BD00ED00E0B9
:100AE00010290020F8B504460126002722460021DF
:100AF000012000F006F805462846FEF77DFD284651
:100B0000F8BDF7B582B005460E46002D01D0012094
:100B100000E00020002802D172B600BFFEE7002EE0
:100B200001D1002701E02F46774338465030FEF7C9
:100B300045FF0446002C09D0204650300190009417
:100B400031462846049B019AFEF765FD204605B014
:100B5000F0BD70B505460E462C46002C02D172B68B
:100B600000BFFEE7FFF75CFD216CE06B48432168A6
:100B7000401860600020A0632068A060E06B401E09
:100B8000216C484321684018E0600021C94344209B
:100B9000015545200155002E10D12069002801D1B2
:100BA000012000E00020002810D12046103000F085
:100BB0002BFC00280AD0FFF795FD07E020461030F7
:100BC000FFF7F6FC20462430FFF7F2FCFFF736FD76
:100BD000012070BDFFB583B006461D46002002907F
:100BE0003446002C02D172B600BFFEE704980028FC
:100BF00002D1206C002801D1012000E00020002853
:100C000002D172B600BFFEE7022D02D1E06B0128CF
:100C100001D1012000E00020002802D172B600BFFF
:100C2000FEE700F0A5FA002802D10598002801D1BE
:100C3000012000E00020002802D172B600BFFEE7CC
:100C400000BFFFF7EDFCA06BE16B884201D3022DE2
:100C50001FD12A4620460499FEF730FC0746606AF9
:100C6000002801D1012000E00020002808D1204602
:100C7000243000F0C9FB002806D0FFF733FD03E065
:100C8000002F01D0FFF72EFDFFF7D8FC012007B0A1
:100C9000F0BD0598002803D1FFF7D0FC0020F6E74F
:100CA0000298002804D16846FFF78CFD01200290CD
:100CB000FFF7C4FCFFF7A6FEFFF7B2FC442108577C
:100CC000401C002802D1002144200155452108572D
:100CD000401C002802D1002145200155FFF7AEFC41
:100CE00005A9684600F0DCF9002819D12046FEF776
:100CF00075FD00280ED0204610300599FFF7DEFD67
:100D00002046FEF7FFFD00F0C3FB002899D1FFF756
:100D1000E9FC96E72046FEF7F5FD00F0B9FB90E709
:100D20002046FEF7EFFD00F0B3FB0020AFE7FFB574
:100D300083B0064617461D463446002C02D172B6D3
:100D400000BFFEE70498002802D1206C002801D1E2
:100D5000012000E00020002802D172B600BFFEE7AB
:100D6000022D02D1E06B012801D1012000E000201A
:100D7000002802D172B600BFFEE7F7F7C7F901906D
:100D8000A06BE16B884201D3022D26D1452001578B
:100D900000912A4620460499FEF790FB0098401CDB
:100DA000002812D1606A002801D1012000E0002053
:100DB00000280FD12046243000F026FB002809D05F
:100DC000002F07D00120386004E00098401C41B299
:100DD000452001550120029001E000200290019879
:100DE000F7F798F9029807B0F0BDF7B584B005465B
:100DF0000E46002003902C46002C02D172B600BF94
:100E0000FEE7002E02D1206C002801D1012000E075
:100E10000020002802D172B600BFFEE700F0A8F95A
:100E2000002802D10698002801D1012000E000200E
:100E3000002802D172B600BFFEE700BFFFF7F0FB4B
:100E4000A76B002F1AD031462046FEF721FB781EF3
:100E5000A0632069002801D1012000E000200028C3
:100E600007D12046103000F0CFFA002801D0FFF75C
:100E700039FCFFF7E3FB012007B0F0BD069800281E
:100E800003D1FFF7DBFB0020F6E70398002804D12D
:100E900001A8FFF797FC01200390FFF7CFFBFFF7B6
:100EA000B1FDFFF7BDFB44210857401C002802D1CB
:100EB00000214420015545210857401C002802D13B
:100EC000002145200155FFF7B9FB06A901A800F054
:100ED000E7F8002819D12046FEF772FC00280ED052
:100EE000204624300699FFF7E9FC2046FEF70AFD6C
:100EF00000F0CEFA0028A1D1FFF7F4FB9EE72046D0
:100F0000FEF700FD00F0C4FA98E72046FEF7FAFC71
:100F100000F0BEFA2046FEF753FC00288ED00020D9
:100F2000AAE7F3B583B00546002002902C460026C0
:100F3000002C02D172B600BFFEE7206C002801D160
:100F4000012000E00020002802D172B600BFFEE7B9
:100F500000F00EF9002802D10498002801D10120E8
:100F600000E00020002802D172B600BFFEE700BFFB
:100F7000FFF756FBA76B002F1CD0781EA0632068DC
:100F8000002802D1FEF7A8FD60602069002801D189
:100F9000012000E00020002807D12046103000F09A
:100FA00033FA002801D0FFF79DFBFFF747FB012034
:100FB00005B0F0BD049800280DD1002E01D101200C
:100FC00000E00020002802D172B600BFFEE7FFF764
:100FD00035FB0020ECE70298002804D16846FFF7B3
:100FE000F1FB01200290FFF729FBFFF70BFDFFF754
:100FF00017FB44210857401C002802D1002144203F
:10100000015545210857401C002802D100214520E8
:101010000155FFF713FB04A9684600F041F80028CA
:1010200024D12046FEF7CCFB002819D020680028E8
:1010300007D1FFF7F5FA606800F094F90646FFF76C
:10104000FDFA204624300499FFF738FC2046FEF7CD
:1010500059FC00F01DFA00288AD1FFF743FB87E70F
:101060002046FEF74FFC00F013FA81E72046FEF71A
:1010700049FC00F00DFA2046FEF7A2FB0028EED056
:10108000002E0BD0FFF7CCFA2046FEF760FA074699
:1010900039466068FFF728FCFFF7D0FA002087E7A1
:1010A00070B505460C46002D02D172B600BFFEE7B2
:1010B000002C02D172B600BFFEE7FFF7B1FA134869
:1010C00002686868131A2068401C002801D10026B5
:1010D00017E00F4928680968884204D06868904280
:1010E00001D801260DE02068984207D92068C01A6F
:1010F00020602846FFF766FB002602E00020206003
:101100000126FFF79BFA304670BD0000E82800205A
:10111000FC280020FFB585B01746B800FEF74EFC4E
:101120000646002E0BD05C20FEF748FC0446002C3F
:1011300001D0266304E03046FFF794FA00E0002473
:10114000002C10D000220F990E986B4613C3039207
:101150003A46089B06990598FEF773FA2046FEF773
:101160001DF9012501E00025ED43284609B0F0BD39
:1011700006490968002901D1012006E004490968EF
:10118000002901D1022000E000207047F028002053
:101190000C2900200149086870470000E828002059
:1011A000F8B50020009042480068002872D14148FC
:1011B0000068451C3F480560002D1CD13E48006872
:1011C0000068002801D1012000E00020002802D1A1
:1011D00072B600BFFEE738480768384800683649ED
:1011E00008603648076036480068401C344908608B
:1011F000FEF738FB00BF3348006885423DD300BF8F
:101200002D4800680068002801D1012000E000207E
:10121000002804D00020C0432A4908602CE026485A
:101220000068C068C4686668B54202D22548066096
:1012300022E0201DFFF750F9A06A002803D02046C5
:101240001830FFF749F92049E06A0968884202D955
:101250001D49E06A08601422E16A51431B4A88185C
:10126000211DFFF7D0F91A49E06A0968C96A884266
:10127000C6D301200090C3E700BF15480068C06ACC
:101280001421484311490858012801D90120009030
:1012900005E0FFE70F480068401C0E4908600E4853
:1012A0000068002801D0012000900098F8BD0000DF
:1012B0000C290020E8280020D8280020DC28002065
:1012C000FC28002004290020EC280020783500208C
:1012D000D4280020F4280020F828002070B5054606
:1012E0002C460026002D35D01B480068844201D1D1
:1012F000012000E00020002802D172B600BFFEE706
:10130000206D002802D172B600BFFEE7206D401E9E
:101310002065E16CE06A88421CD0206D002819D15C
:10132000201DFFF7D9F8E06CE0620721E06A081A97
:10133000A0610A49E06A0968884202D90749E06A5F
:1013400008601422E16A5143054A8818211DFFF7FD
:101350005AF90126304670BDD4280020EC28002020
:101360007835002070B505462C460026002D42D069
:101370002249E06A0968C96A884235D2A069C00F6B
:10138000C007002805D11D480068C06A0721081A57
:10139000A0611422E06A5043194A801861698142B1
:1013A00001D1012000E00020002817D0201DFFF708
:1013B00093F812480068C06AE0621249E06A09685E
:1013C000884202D90F49E06A08601422E16A514359
:1013D0000B4A8818211DFFF716F903E0074800683B
:1013E000C06AE062012606E00449E06C0968C96A47
:1013F000884200D20126304670BD0000D42800206B
:1014000078350020EC28002070B50646F068C468E6
:10141000002C02D172B600BFFEE720461830FFF75D
:101420005BF815480068002813D1201DFFF754F819
:101430001249E06A0968884202D91049E06A0860E6
:101440001422E16A51430E4A8818211DFFF7DBF888
:1014500004E0214618310B48FFF7D5F80A49E06A45
:101460000968C96A884204D9012501200749086032
:1014700000E00025284670BD0C290020EC28002043
:10148000783500202C360020D4280020F8280020B1
:1014900070B50024002632480068002802D172B6D8
:1014A00000BFFEE7FFF7BCF82D480068401E2C493E
:1014B00008600846006800284DD12A4800680028C6
:1014C00049D022E02848C068C46820461830FFF799
:1014D00003F8201DFFF700F82449E06A09688842F4
:1014E00002D92249E06A08601422E16A5143204A85
:1014F0008818211DFFF787F81E49E06A0968C96A44
:10150000884202D301201C4908601748006800285F
:1015100001D1012000E000200028D3D0002C01D010
:10152000FEF7A0F915480568002D0DD000BFFFF7A4
:1015300037FE002802D001200F4908606D1E002DE3
:10154000F5D100200D4908600B480068002802D042
:101550000126FFF7C7F8FFF771F8304670BD0000AD
:101560000C290020E42800202C360020EC28002044
:1015700078350020D4280020F8280020F428002006
:1015800040BA7047C0BA70470138FDD170470000BB
:10159000F7B50325AD06286A82B016460C4640080A
:1015A00040002862286A022108432862286A8007CE
:1015B000FCD46620686001272F61A86AC005FCD5AD
:1015C000992068602F61A86AC005FCD5FF20913082
:1015D000FFF7DAFFFF230133AB626846EF60352186
:1015E00069602F61A96AC905FCD5AB62A969EF6082
:1015F000C9B205226A602F61AA6AD205FCD5AB6226
:10160000AA690902D2B211430180C80702D003209F
:1016100005B0F0BDAB626869FF210831884368619D
:101620006869C91E08436861029800024830686012
:101630000820A860EE602F61A86AC005FCD5FF20D5
:101640000130A8620023F61CB0080ED0B208114881
:10165000006899006054060A09194E70060C000EC5
:101660008E705B1CC8709A42F1D8FF200130A862CE
:101670006869FF2108318843686168693843686197
:10168000286A800880002862286A3843286200207F
:1016900005B0F0BD8000000C032080064169FF22E8
:1016A000083291434161426901210A434261026A61
:1016B000920892000262026A0A43026270470000C6
:1016C000002003218906096A49084900032292067D
:1016D00011621146096A0222114303229206116225
:1016E00000BF03218906096A022211400229F8D0AD
:1016F000D1010322920691620321D1609F215160A2
:101700000121116100BF03218906896AFF2201328C
:1017100011409142F7D103229206916211468869E5
:101720004969FF2208329143032292065161114612
:101730004969012211430322920651611146096A47
:101740008908890011621146096A012211430322A6
:1017500092061162704700000000000001020304BD
:10176000000001020138FDD170470000F0B40324ED
:10177000A406236A5B085B002362236A02252B43CD
:101780002362236A9B07FCD4FF230133A3626569AC
:10179000DE1DB543656165691E1D35436561000247
:1017A0006B3060600820A060E26001262661A06ABC
:1017B000C005FCD5A3620023D21C90080ED095086A
:1017C0000F4800689A008854070A52185770070C8F
:1017D000000E97705B1CD0709D42F1D86069FF21AC
:1017E000083188436061606930436061206A800825
:1017F00080002062206A30432062F0BC00207047E5
:101800008000000CF8B5064601200025C004864281
:1018100001D90520F8BD0324A406206A4008400031
:101820002062206A022108432062206A8007FCD4DB
:10183000FF270137A76200F0BBF8002801D003257D
:1018400015E00620606001212161A06AC005FCD579
:10185000A7623002203060602161A06AC005FCD51B
:10186000A7620C4800F0C8F8002800D10225606982
:10187000FF2108318843606160690121084360618C
:10188000206A800880002062206A0843206228467F
:10189000F8BD0000E6960100F7B506460120C00439
:1018A00082B01546864202D9052005B0F0BD03205E
:1018B0008006016A490849000162016A0222114357
:1018C0000162016A8907FCD4FF2101318162F2B211
:1018D0008C1AA54200D8ACB20398009000F068F8CA
:1018E000002840D106214806416001210161816A3A
:1018F000C905FCD5FF2101310320800681624169C1
:10190000FF22083291434161416904221143416140
:10191000310232314160C4600022002C16D9009897
:1019200087183B78F87819467B7800061B02194324
:10193000BB781B04194301430802F978000A090621
:10194000084319490860121DA242E8D3012103206F
:1019500080060161816AC905FCD5FF2101318162E0
:10196000124800F049F8A54209D003983619001929
:101970002D1BFF2401340390A542ADD8ABE7032013
:1019800080064169FF220832914341614169012289
:1019900011434161016A890889000162016A1143AA
:1019A0000162002005B0F0BD8000000C1A060000A6
:1019B00038B40125032080066A46C56035214160A0
:1019C0000561816AC905FCD5FF24013484628169FF
:1019D000C560CBB2052141600561816AC905FCD5AE
:1019E000846280691902C0B2014388B21180C007C5
:1019F00000D0012038BC7047F8B400210125032233
:101A000092066B46D560352454601561946AE405EE
:101A1000FCD5FF27013797629469D560E4B20526AB
:101A200056601561966AF605FCD5976296692402A0
:101A3000F6B234431C80E30722D0814202D9F8BCBD
:101A400000207047032292066B46D560352454600F
:101A50001561491C946AE405FCD597629469D560C8
:101A6000E4B2052656601561966AF605FCD59762C4
:101A700092692402D2B21443A2B21C80D207DCD1F4
:101A8000F8BC012070470000001713001710001762
:101A90000E0017090017040017000017180117148B
:101AA0000117150117190000F7B586B00020029044
:101AB0005C48154604695C480E46824201D90546D9
:101AC00002E0002D00D10125002C08D0A188069845
:101AD000814204D1E088B04201D1012002905348F4
:101AE000039084460698010431430020002C1CD04A
:101AF0000A0CA7888BB2974207D1E7889F4204D18E
:101B0000002807D02168016007E020462468002CE7
:101B1000EFD10AE0614622680A602168002902D0FC
:101B20000020206001E061464860002C07D10221BE
:101B3000102000F095F8069981800446C68028019F
:101B4000052100F077F807467D200E464643EFF367
:101B50001085012080F31088684600F087F885F32F
:101B6000108800980490C0190501019927202D09BB
:101B70008E1900010591864203D96D1C2D012D0996
:101B8000361AE660A5600398294F864600208446F1
:101B900070460068002813D0A268E1680091C3680D
:101BA00081680193531A1B011B09BB420AD291425F
:101BB00003D1019A0099914204D984460068E9E76B
:101BC0007246546020606046002801D0046001E045
:101BD00071460C60134802990069002901D1A042A6
:101BE00003D1C168806800F047F8EFF3108401204A
:101BF00080F3108802A800F039F884F31088039964
:101C000002980191291A090109090090B94204D2E8
:101C1000A84205D10198864202D8032000F032F88C
:101C200009B0F0BDC8010020FFFF7F02D8010020ED
:101C3000FFFFFF0730B50B4601460020202201249C
:101C400009E00D46D5409D4205D31D469540491BF0
:101C50002546954040191546521E002DF1DC30BD39
:101C600003B40148019001BD2D7A010003B401487D
:101C7000019001BD5DB6020003B40148019001BDB1
:101C80009DB6020003B40148019001BDAD7801008A
:101C900030B4C36882688868084D141A2401C96882
:101CA0002409AC4203D2904204D18B4202D830BC0A
:101CB0000120704730BC002070470000FFFFFF0785
:101CC0000A0C838889B2934204D1C088884201D12A
:101CD000012070470020704770B40546006800225C
:101CE000002810D00B0C86888CB29E4207D1C68883
:101CF000A64204D10168002A07D0116006E002461E
:101D000000680028EFD170BC704729600168002985
:101D100003D00021016070BC70476A6070BC7047DE
:101D2000F0B5104F026886460025002A10D0C8681A
:101D30008C6893688446E01A00010009D668B842AE
:101D400008D2A34201D1B44504D915461268ECE784
:101D5000704641600A60002D01D02960F0BD7046D8
:101D60000160F0BDFFFFFF0770B584B004460E466A
:101D7000EFF31085012080F3108802A8FFF776FFAB
:101D800085F3108802980399024600900191A01AE9
:101D9000000107490009884204D2A24205D10198F6
:101DA000864202D8012004B070BD002004B070BD8E
:101DB000FFFFFF0730B583B00446EFF31085012025
:101DC00080F310886846FFF751FF85F3108801996A
:101DD00000986160206003B030BD0000AFFD0001DD
:101DE00011FD0001B9FC000161FC0001130C0000B1
:101DF000CDD10001150C0000E5D20001170C000048
:101E000015D00001000C000061D000010647000061
:101E1000DFFF000103470000BB000101084700008D
:101E200009FF00010E470000A9FB00010547000063
:101E3000E100010100171300171000170E00170929
:101E400000170400170000171801171401171501D7
:101E500017190000F7B586B0002002905C481546BF
:101E600004695C480E46824201D9054602E0002D15
:101E700000D10125002C08D0A1880698814204D108
:101E8000E088B04201D1012002905348039084467B
:101E90000698010431430020002C1CD00A0CA788AE
:101EA0008BB2974207D1E7889F4204D1002807D020
:101EB0002168016007E020462468002CEFD10AE089
:101EC000614622680A602168002902D00020206053
:101ED00001E061464860002C07D10221102000F08B
:101EE00095F8069981800446C6802801052100F0F6
:101EF00077F807467D200E464643EFF31085012014
:101F000080F31088684600F087F885F31088009801
:101F10000490C0190501019927202D098E1900018F
:101F20000591864203D96D1C2D012D09361AE660F4
:101F3000A5600398294F86460020844670460068B5
:101F4000002813D0A268E1680091C36881680193FA
:101F5000531A1B011B09BB420AD2914203D1019AB9
:101F60000099914204D984460068E9E772465460BA
:101F700020606046002801D0046001E071460C60DA
:101F8000134802990069002901D1A04203D1C16818
:101F9000806800F047F8EFF31084012080F3108888
:101FA00002A800F039F884F310880399029801918F
:101FB000291A090109090090B94204D2A84205D1A1
:101FC0000198864202D8032000F032F809B0F0BD33
:101FD000C8010020FFFF7F02D8010020FFFFFF079C
:101FE00030B50B46014600202022012409E00D46B1
:101FF000D5409D4205D31D469540491B2546954039
:1020000040191546521E002DF1DC30BD03B40148C5
:10201000019001BD2D7A010003B40148019001BD7A
:102020005DB6020003B40148019001BD9DB60200F7
:1020300003B40148019001BDAD78010030B4C3681C
:1020400082688868084D141A2401C9682409AC42C2
:1020500003D2904204D18B4202D830BC0120704799
:1020600030BC002070470000FFFFFF070A0C838888
:1020700089B2934204D1C088884201D101207047BF
:102080000020704770B4054600680022002810D078
:102090000B0C86888CB29E4207D1C688A64204D11A
:1020A0000168002A07D0116006E002460068002897
:1020B000EFD170BC704729600168002903D000216E
:1020C000016070BC70476A6070BC7047F0B5104F1B
:1020D000026886460025002A10D0C8688C6893687C
:1020E0008446E01A00010009D668B84208D2A3422B
:1020F00001D1B44504D915461268ECE77046416039
:102100000A60002D01D02960F0BD70460160F0BD6D
:10211000FFFFFF0770B584B004460E46EFF310854D
:10212000012080F3108802A8FFF776FF85F310885E
:1021300002980399024600900191A01A00010749F4
:102140000009884204D2A24205D10198864202D8F1
:10215000012004B070BD002004B070BDFFFFFF0778
:1021600030B583B00446EFF31085012080F310886A
:102170006846FFF751FF85F3108801990098616068
:10218000206003B030BD00000017130017100017C7
:102190000E00170900170400170000171801171484
:1021A0000117150117190000F7B586B0002002903D
:1021B0005C48154604695C480E46824201D90546D2
:1021C00002E0002D00D10125002C08D0A18806983E
:1021D000814204D1E088B04201D1012002905348ED
:1021E000039084460698010431430020002C1CD043
:1021F0000A0CA7888BB2974207D1E7889F4204D187
:10220000002807D02168016007E020462468002CE0
:10221000EFD10AE0614622680A602168002902D0F5
:102220000020206001E061464860002C07D10221B7
:10223000102000F095F8069981800446C680280198
:10224000052100F077F807467D200E464643EFF360
:102250001085012080F31088684600F087F885F328
:10226000108800980490C0190501019927202D09B4
:102270008E1900010591864203D96D1C2D012D098F
:10228000361AE660A5600398294F864600208446EA
:1022900070460068002813D0A268E1680091C36806
:1022A00081680193531A1B011B09BB420AD2914258
:1022B00003D1019A0099914204D984460068E9E764
:1022C0007246546020606046002801D0046001E03E
:1022D00071460C60134802990069002901D1A0429F
:1022E00003D1C168806800F047F8EFF31084012043
:1022F00080F3108802A800F039F884F3108803995D
:1023000002980191291A090109090090B94204D2E1
:10231000A84205D10198864202D8032000F032F885
:1023200009B0F0BDC8010020FFFF7F02D8010020E6
:10233000FFFFFF0730B50B46014600202022012495
:1023400009E00D46D5409D4205D31D469540491BE9
:102350002546954040191546521E002DF1DC30BD32
:1023600003B40148019001BD2D7A010003B4014876
:10237000019001BD5DB6020003B40148019001BDAA
:102380009DB6020003B40148019001BDAD78010083
:1023900030B4C36882688868084D141A2401C9687B
:1023A0002409AC4203D2904204D18B4202D830BC03
:1023B0000120704730BC002070470000FFFFFF077E
:1023C0000A0C838889B2934204D1C088884201D123
:1023D000012070470020704770B405460068002255
:1023E000002810D00B0C86888CB29E4207D1C6887C
:1023F000A64204D10168002A07D0116006E0024617
:1024000000680028EFD170BC70472960016800297E
:1024100003D00021016070BC70476A6070BC7047D7
:10242000F0B5104F026886460025002A10D0C86813
:102430008C6893688446E01A00010009D668B842A7
:1024400008D2A34201D1B44504D915461268ECE77D
:10245000704641600A60002D01D02960F0BD7046D1
:102460000160F0BDFFFFFF0770B584B004460E4663
:10247000EFF31085012080F3108802A8FFF776FFA4
:1024800085F3108802980399024600900191A01AE2
:10249000000107490009884204D2A24205D10198EF
:1024A000864202D8012004B070BD002004B070BD87
:1024B000FFFFFF0730B583B00446EFF3108501201E
:1024C00080F310886846FFF751FF85F31088019963
:1024D00000986160206003B030BD00000028000259
:1024E000000000000328000200000000002A000A8B
:1024F000008020000328000200000000012A0002E2
:10250000008002000328000200000000042A0002EC
:10251000008008000328000200000000A62A000234
:10252000008001000328000200000000C92A000208
:1025300000800100002800020000000003280002C3
:1025400000000000052A0020008004000229000A83
:10255000000002000328000200000000292B000AEE
:102560000080100003280002000000002A2B000257
:1025700000801000FFFF0000ADB00001A40D0000BE
:1025800029C90001A50D000069C900011A0D00004C
:10259000C5CF0001150D0000E5C90001000D0000C8
:1025A00015CA00011C0D0000E3CF0001A70D0000BB
:1025B000DDCE0001A80D000001D00001020C0000DA
:1025C00061D10001000C0000F1D00001010E0000FB
:1025D000F1C300010F0E000041C80001110E000000
:1025E000B1C800012C0E00001DC80001030E000040
:1025F0008DC500010A0E000065C70001300E000005
:1026000009C800010C0E0000E5C80001000E000022
:1026100011C30001090E000071C30001010F000089
:102620007DB10001020F0000F5AE0001030F0000B4
:1026300055B10001040F0000B9E700017425010144
:102640008014002001001900001713001710001754
:102650000E001709001704001700001718011714BF
:102660000117150117190000F7B586B00020029078
:102670005C48154604695C480E46824201D905460D
:1026800002E0002D00D10125002C08D0A188069879
:10269000814204D1E088B04201D101200290534828
:1026A000039084460698010431430020002C1CD07E
:1026B0000A0CA7888BB2974207D1E7889F4204D1C2
:1026C000002807D02168016007E020462468002C1C
:1026D000EFD10AE0614622680A602168002902D031
:1026E0000020206001E061464860002C07D10221F3
:1026F000102000F095F8069981800446C6802801D4
:10270000052100F077F807467D200E464643EFF39B
:102710001085012080F31088684600F087F885F363
:10272000108800980490C0190501019927202D09EF
:102730008E1900010591864203D96D1C2D012D09CA
:10274000361AE660A5600398294F86460020844625
:1027500070460068002813D0A268E1680091C36841
:1027600081680193531A1B011B09BB420AD2914293
:1027700003D1019A0099914204D984460068E9E79F
:102780007246546020606046002801D0046001E079
:1027900071460C60134802990069002901D1A042DA
:1027A00003D1C168806800F047F8EFF3108401207E
:1027B00080F3108802A800F039F884F31088039998
:1027C00002980191291A090109090090B94204D21D
:1027D000A84205D10198864202D8032000F032F8C1
:1027E00009B0F0BDC8010020FFFF7F02D801002022
:1027F000FFFFFF0730B50B460146002020220124D1
:1028000009E00D46D5409D4205D31D469540491B24
:102810002546954040191546521E002DF1DC30BD6D
:1028200003B40148019001BD2D7A010003B40148B1
:10283000019001BD5DB6020003B40148019001BDE5
:102840009DB6020003B40148019001BDAD780100BE
:1028500030B4C36882688868084D141A2401C968B6
:102860002409AC4203D2904204D18B4202D830BC3E
:102870000120704730BC002070470000FFFFFF07B9
:102880000A0C838889B2934204D1C088884201D15E
:10289000012070470020704770B405460068002290
:1028A000002810D00B0C86888CB29E4207D1C688B7
:1028B000A64204D10168002A07D0116006E0024652
:1028C00000680028EFD170BC7047296001680029BA
:1028D00003D00021016070BC70476A6070BC704713
:1028E000F0B5104F026886460025002A10D0C8684F
:1028F0008C6893688446E01A00010009D668B842E3
:1029000008D2A34201D1B44504D915461268ECE7B8
:10291000704641600A60002D01D02960F0BD70460C
:102920000160F0BDFFFFFF0770B584B004460E469E
:10293000EFF31085012080F3108802A8FFF776FFDF
:1029400085F3108802980399024600900191A01A1D
:10295000000107490009884204D2A24205D101982A
:10296000864202D8012004B070BD002004B070BDC2
:10297000FFFFFF0730B583B00446EFF31085012059
:1029800080F310886846FFF751FF85F3108801999E
:1029900000986160206003B030BD0000FFFF0000C0
:1029A00047B30001130E0000B5C00001150E000072
:1029B000A1BF0001170E000031C60001190E000072
:1029C00001C600019C290101050000000017130049
:1029D000171000170E001709001704001700001742
:1029E000180117140117150117190000F7B586B063
:1029F000002002905C48154604695C480E468242FD
:102A000001D9054602E0002D00D10125002C08D097
:102A1000A1880698814204D1E088B04201D101200A
:102A200002905348039084460698010431430020E5
:102A3000002C1CD00A0CA7888BB2974207D1E788DC
:102A40009F4204D1002807D02168016007E020469A
:102A50002468002CEFD10AE0614622680A602168F0
:102A6000002902D00020206001E061464860002C6F
:102A700007D10221102000F095F8069981800446C4
:102A8000C6802801052100F077F807467D200E4614
:102A90004643EFF31085012080F31088684600F06C
:102AA00087F885F3108800980490C01905010199F2
:102AB00027202D098E1900010591864203D96D1C2E
:102AC0002D012D09361AE660A5600398294F864628
:102AD0000020844670460068002813D0A268E16890
:102AE0000091C36881680193531A1B011B09BB4203
:102AF0000AD2914203D1019A0099914204D98446A5
:102B00000068E9E77246546020606046002801D002
:102B1000046001E071460C601348029900690029C5
:102B200001D1A04203D1C168806800F047F8EFF3FB
:102B30001084012080F3108802A800F039F884F393
:102B40001088039902980191291A09010909009036
:102B5000B94204D2A84205D10198864202D8032086
:102B600000F032F809B0F0BDC8010020FFFF7F027D
:102B7000D8010020FFFFFF0730B50B4601460020BB
:102B80002022012409E00D46D5409D4205D31D4673
:102B90009540491B2546954040191546521E002D6B
:102BA000F1DC30BD03B40148019001BD2D7A010074
:102BB00003B40148019001BD5DB6020003B40148B1
:102BC000019001BD9DB6020003B40148019001BD12
:102BD000AD78010030B4C36882688868084D141A63
:102BE0002401C9682409AC4203D2904204D18B422B
:102BF00002D830BC0120704730BC00207047000074
:102C0000FFFFFF070A0C838889B2934204D1C08872
:102C1000884201D1012070470020704770B40546FA
:102C200000680022002810D00B0C86888CB29E42CF
:102C300007D1C688A64204D10168002A07D01160D6
:102C400006E0024600680028EFD170BC704729609A
:102C50000168002903D00021016070BC70476A60E0
:102C600070BC7047F0B5104F026886460025002AF8
:102C700010D0C8688C6893688446E01A0001000987
:102C8000D668B84208D2A34201D1B44504D915464A
:102C90001268ECE7704641600A60002D01D029609F
:102CA000F0BD70460160F0BDFFFFFF0770B584B056
:102CB00004460E46EFF31085012080F3108802A829
:102CC000FFF776FF85F3108802980399024600907B
:102CD0000191A01A000107490009884204D2A242CA
:102CE00005D10198864202D8012004B070BD0020B1
:102CF00004B070BDFFFFFF0730B583B00446EFF3AB
:102D00001085012080F310886846FFF751FF85F396
:102D10001088019900986160206003B030BD000008
:102D200010CA000011CA114B008011CA11CA11CA81
:102D3000002800000000000000000000000000006B
:102D40000002000000000328000000000000000056
:102D5000000000000000000A0000000011CA00008E
:102D600011CA114B008011CA11CA11CA000400C057
:102D70000002012900000000000000000000000027
:102D80000000000A0080140003280000000000007A
:102D90000000000000000000000A0000000012CA4D
:102DA000000011CA114B008011CA11CA11CA0010CB
:102DB00000C0000202290000000000000000000026
:102DC00000000000000A008014000000044700001A
:102DD0008DBE00010A47000031BE00010747000018
:102DE00021BE0001CC2D0101030000000100000004
:102DF000000000000200000000000000982F010108
:102E0000A02F0101BD8D00017C2F0101642F010164
:102E1000D9900001902F0101C42E0101E58F00011E
:102E2000602F0101902E0101398F0001302F010127
:102E3000002F0101498E0001842F0101342F01016F
:102E4000258C00015B424C455D20727769702068DB
:102E50006561702063656C6C733A20656E763D2504
:102E600030386C582F25752064623D2530386C58F9
:102E70002F2575206D73673D2530386C582F2575CB
:102E8000206E7265743D2530386C582F25750A0008
:102E90006C6F67205B6F6E7C6F66665D3A20616366
:102EA00074697665207072696E74696E67207377D5
:102EB00069746368202864656661756C74206F6648
:102EC0006629000073686F77204672656552544F1B
:102ED000532072756E74696D6520696E666F202867
:102EE000757074696D652F7461736B732F6865619C
:102EF000702F7461736B206C69737429000000007B
:102F00006C6564203C317C323E203C6F6E7C6F6689
:102F1000667C746F67676C653E3A20636F6E74728F
:102F20006F6C20626F617264204C454400000000A9
:102F30006C65640073686F772072756E6E696E677A
:102F40002062616E6B20616E6420626F6F747365C6
:102F50007474696E67207265636F726400000000AC
:102F60006C6F670073686F77206669726D77617246
:102F7000652076657273696F6E0000007665727306
:102F8000696F6E0062616E6B696E666F00000000B3
:102F9000737973696E666F0068656C70000000007D
:102FA0006C69737420616C6C20636F6D6D616E640D
:102FB00073000000D42F01010000002068290000E8
:102FC0002288000168360101682900202081000064
:102FD000F02A00000006390090D0030001103611DD
:102FE000D80D490868496813F008FB0498EFF78E7C
:102FF000FF0446C1888088FF22FFF79DFD2046FF21
:10300000F73AFCB3E705B0F0BD0000FFFFFF07D8BB
:10301000010020C804202930D70200004B1847FBCC
:10302000FD06460520307075800099B181301D394C
:1030300046E5F773FD3046F9F70EFF0E22294642AA
:10304000200445FD074030112E0CD0534B052203C0
:10305000212846FDF733FE121E40274B75002D0533
:10306000D0398F002902D00099897900E000211120
:1030700076FAF74BF8044D2859F9F7FBFE002028A3
:1030800051801006000400200777107838B5049CA2
:103090000094014CA04738BD5143F84A26468F188A
:1030A00039462036FD6D707D80311191C97FA03782
:1030B0000E912246397815320F92F14A1092032967
:1030C0002BD0002873D0F17D0F980CF00DF800285C
:1030D0006FD0688869460883F0B597B008780C46C9
:1030E0000F90002014900F9848214843FE49224633
:1030F0004018064680361090F17F0091C56DA030D3
:103100001690014E100A274612922037F74A1552A0
:10311000146C2AD061783C2949D0432947D0787D66
:1031200000287DD0F97D129800F0FCF9002878D0B5
:10313000698868468184687A297A0004090208430C
:10314000E97908430690A97A08A84172E97A817260
:10315000297BC17229460D310E380E9100F02FFAED
:10316000A878400733D5002132E0907E012806D0B0
:10317000507E401E0006000E507603D00614300428
:10318000DB480106141200F0D2F9169A01211170E1
:10319000A978D448C9075C369026482359430818B3
:1031A0000022A0300270FF20F07752E0012202706E
:1031B000A878CC49C0074CD00098482358434020F9
:1031C000101442E0E97C08A80173297D4173697DF0
:1031D0008173A97DC108100D0174297E4174697E37
:1031E0008174B189BC102281F189C181318A018247
:1031F000109940318A8F8283C98F0184B188C1833D
:10320000F18841840021C18442241472B848817835
:1032100008A8C17401E04DE11BE002260675C82133
:10322000CC140C02D4E87A800705D5297B0E143023
:103230000A7EF908A9087503A90F0C1412002801C9
:10324000D11698067060783C2870D030E1628A14FC
:103250003D0A82A2884A82A2790A75E2794A7520DB
:103260007A8875E07EC875A08B0883E08B48832040
:103270008C8883608CC8832146243108A800F0A480
:10328000F9787A08A94871B87A8871A08DC81405B0
:1032900085206B0BC210050C90012018103F75386B
:1032A0007D0875B87D8875A878C006C017401CC811
:1032B000758E486946028A0A87428A4A87827D0853
:1032C000A90A77C27D4A77027E8A77428B10A90AC3
:1032D00080828B4A80807F087104A900A438043260
:1032E000F9000A14487C49401803907C3012990078
:1032F000F05DF90398F97D8030817003990922A06F
:10330000310A700121C170039800218166E18B4967
:103310000041660521C166016715996030C97E00CC
:103320002904D072498161012102E02ABA48098149
:103330006181750099818224400DF6F8022802D23D
:10334000012100F003F912201B05F906280CD20A0E
:10335000215F4A41438918FF318131497F89070341
:10336000D5FA7D7C23FCF8961005FFF81699E03518
:10337000C41A01AE1818092000F0FBF821460F31DD
:10338000059100284ED020233E22002156241C0601
:10339000F6F806460A96031714986C2012D00020FF
:1033A00000E03C2070700120307100987080162081
:1033B000052CD0B01D5A2407F2F8F87D7071AC20AE
:1033C0001306D52146304609310C3000F0E7F803EA
:1033D000E030460A12DD2025C810063046123005BE
:1033E0003032DA1A12121A1406D0F8E08B309A161C
:1033F000709A2813B083B87AB077304600F0BFF8DF
:103400003AE0287B7071DC2007B01D00F0C2F8168E
:103410003006B4F83DE0149E1A2EC23008A7F80119
:10342000210646019E120D9E300470703198200BCB
:10343000F87D820709D57171B01D6A3004A5F80ABC
:10344000B6400B30461DE0C007C00F7071B2129934
:1034500078100BB081208CF081608C3082782274DF
:1034600062300483F80660121660302477F8142165
:10347000017000994180B97D017100F075F81598CF
:10348000807E022826D160781499084322D0082C27
:10349000120B2C100461F8122C1C0C61784170295D
:1034A0007881700FE0406404100AC00600200A20F2
:1034B0000000390412400C1D88031C0820B1A20131
:1034C00000041131051007998180397E81563C0630
:1034D0004AF80020171805100640BA7047C004606B
:1034E0000D03B40148019001BD919B02000C83E1E2
:1034F000980C837D9F0C700449FA010C8309D30C4E
:10350000836D5B24933D99488290488355073083AF
:10351000D59C3083397B181027796D01000021017B
:10352000804180818070470A7802704B7843708AAE
:10353000788270CA78C2700B7903714A7942711A25
:1035400020046802600E0F34704740063414497B33
:1035500041700570F1F7F3FC2068F1F7A4FB2560DA
:1035600003141B2400761C0980024080C10240061F
:103570002B061C19F8B54E784821F0B24843234970
:10358000214D41180C46AA7EA03400275406A2FF04
:10359000500EFFA0C0060DFFC0060DFFC0060DFFB8
:1035A000C0060DFFC0060DFFC0060DA7C0066DE8E2
:1035B000072C22EDC3020010B5074CE06900040897
:1035C000D5FFF7F3FF05480078002802D10120C09D
:1035D00003206210C00C1D100722C6580149010DBE
:1035E000FF00070DFF00070DFF00070DFF00070D8F
:1035F000FF00070DFF00070D7800070C05FF000016
:10360000F401C0060DFFC0060DFFC0060DFFC00689
:103610000DFFC0060DFFC0060DB6C0060C05380034
:1036200000C202940D0DFFC0060DFFC0060DFFC0C5
:10363000060DFFC0060DFFC0060DFFC0060D7CC0C5
:10364000060DFF800D0DFFC0060DFFC0060DFFC06B
:10365000060DFFC0060DFFC0060DF4C006ED90225A
:0836600012AA01025100010051
:00000001FF
